:0200000480007A
:10000000B72F0000938F0F8073900F306F00400365
:100010001300000013000000130000001300000094
:100020001300000013000000130000001300000084
:100030001300000013000000130000001300000074
:100040009702000093824211739052309300000097
:10005000130100009301000013020000930200004E
:100060001303000093030000130400009304000036
:10007000130500009305000013060000930600001E
:100080001307000093070000130800009308000006
:100090001309000093090000130A0000930A0000EE
:1000A000130B0000930B0000130C0000930C0000D6
:1000B000130D0000930D0000130E0000930E0000BE
:1000C000130F0000930F000097110200938141D09D
:1000D0001705020013050553979503009385457294
:1000E00013060000EF00001A170502001305C545AE
:1000F000970502009385654D13060000EF008018F8
:1001000017A503001305057097B503009385456F88
:1001100037B6ABAB1306B6BAEF00C01617B1030083
:100120001301416EEF80D0249392120093D21200FB
:100130009382D2FF638A02008322010013014100EF
:100140006F0000177300203083220100130141006B
:10015000730020301301C1FF23205100F32220340B
:10016000E3C402FC8322010013014100130141F8A2
:1001700023221100232421002326310023284100BB
:10018000232A5100232C6100232E71002320810299
:10019000232291022324A1022326B1022328C10293
:1001A000232AD102232CE102232EF1022320010570
:1001B0002322110523242105232631052328410567
:1001C000232A5105232C6105232E71052320810745
:1001D000232291072324A1072326B1072328C1073F
:1001E000232AD107232CE107232EF107732520347E
:1001F000F3251034130601006F000000731015344E
:1002000083204100032181008321C10003220101D9
:1002100083224101032381018323C10103240102BD
:1002200083244102032581028325C10203260103A1
:1002300083264103032781038327C1030328010485
:1002400083284104032981048329C104032A010569
:10025000832A4105032B8105832BC105032C01064D
:10026000832C4106032D8106832DC106032E010731
:10027000832E4107032F8107832FC1071301C10775
:10028000730020302320C5006376B50013054500B8
:100290006FF05FFF678000000000000000000000BA
:1002A000000000000000000000000000000000004E
:1002B000130101F8232011002322210023243100FF
:1002C0002326410023285100232A6100232C71009A
:1002D000232E8100232091022322A1022324B10294
:1002E0002326C1022328D102232AE102232CF10272
:1002F000232E010323201105232221052324310568
:100300002326410523285105232A6105232C710545
:10031000232E8105232091072322A1072324B1073F
:100320002326C1072328D107232AE107232CF1071D
:100330009702020083A2822423A02200F322103419
:10034000232E5106EF00C03B1701020003210123B9
:10035000032101008322C10773901234B7220000E9
:100360009382028873A00230832001000322C1001F
:100370008322010103234101832381010324C1015D
:100380008324010203254102832581020326C10241
:100390008326010303274103832781030328C10325
:1003A000832801040329410483298104032AC10409
:1003B000832A0105032B4105832B8105032CC105ED
:1003C000832C0106032D4106832D8106032EC106D1
:1003D000832E0107032F4107832F81071301010893
:1003E00073002030970202009382C22123A01200E2
:1003F00023A2220023A4320023A6420023A85200F5
:1004000023AA620023AC720023AE820023A09202D2
:1004100023A2A20223A4B20223A6C20223A8D202CC
:1004200023AAE20223ACF20223AE020323A01205A8
:1004300023A2220523A4320523A6420523A85205A0
:1004400023AA620523AC720523AE820523A092077E
:1004500023A2A20723A4B20723A6C20723A8D20778
:1004600023AAE20723ACF207EF60506E17010200E7
:100470000321C110032101008322C10773901234AC
:10048000B72200009382028873A00230832001000B
:100490000322C1008322010103234101832381013F
:1004A0000324C10183240102032541028325810223
:1004B0000326C10283260103032741038327810307
:1004C0000328C103832801040329410483298104EB
:1004D000032AC104832A0105032B4105832B8105CF
:1004E000032CC105832C0106032D4106832D8106B3
:1004F000032EC106832E0107032F4107832F810797
:100500001301010873002030970202009382820FCA
:1005100083A0020003A1420083A1820003A2C200C3
:1005200083A2020103A3420183A3820103A4C201A7
:1005300083A4020203A5420283A5820203A6C2028B
:1005400083A6020303A7420383A7820303A8C2036F
:1005500083A8020403A9420483A9820403AAC20453
:1005600083AA020503AB420583AB820503ACC20537
:1005700083AC020603AD420683AD820603AEC2061B
:1005800083AE020703AFC20983AF82076780000012
:1005900073700430130101F823201100232221007D
:1005A000232431002326410023285100232A6100FF
:1005B000232C7100232E8100232091022322A102EB
:1005C0002324B1022326C1022328D102232AE102D7
:1005D000232CF102232E01032320110523222105C0
:1005E000232431052326410523285105232A6105AB
:1005F000232C7105232E8105232091072322A10797
:100600002324B1072326C1072328D107232AE10782
:10061000232CF1079702020083A242F623A02200B6
:10062000232E1106EF30406F17010200032101F560
:10063000032101008322C10773901234B722000006
:100640009382028873A00230832001000322C1003C
:100650008322010103234101832381010324C1017A
:100660008324010203254102832581020326C1025E
:100670008326010303274103832781030328C10342
:10068000832801040329410483298104032AC10426
:10069000832A0105032B4105832B8105032CC1050A
:1006A000832C0106032D4106832D8106032EC106EE
:1006B000832E0107032F4107832F810713010108B0
:1006C00073002030737004306F00000073104530E9
:1006D000678000007325403073F04330678000006E
:1006E00097070000938747FE232EB5FE2322C5FA05
:1006F000232635F82320F5F8130505F86780000058
:10070000130101FF23261100EF609041EF20D01864
:10071000631805008320C1001301010167800000F8
:100720008320C100130101016F30005F9307850032
:100730001307F0FF2322F5002324E5002326F5000C
:100740002328F500232005006780000023280500EA
:10075000678000008327450023A2F50003A78700D8
:1007600023A4E50003A787002322B70023A4B70032
:1007700023A8A50083270500938717002320F500F1
:100780006780000003A605009307F0FF13078500AC
:100790006316F6006F008003138707008327470066
:1007A00083A60700E37AD6FE23A2F50023A4B700B0
:1007B00023A4E5002322B70023A8A5008327050072
:1007C000938717002320F5006780000003270501A9
:1007D000832747006FF05FFD0327450083268500D0
:1007E000832705012324D70003278500832645009E
:1007F0002322D70003A747006316A700032785001D
:1008000023A2E7002328050003A507001305F5FF31
:1008100023A0A70067800000032605049387050036
:10082000630406028325C50003274500B385C50080
:100830002326B50063E6E500832505002326B500E1
:10084000138507006F50100A67800000130101FF35
:100850002324810023261100130405002322910084
:10086000EF30D07F83278404635AF0048327440247
:1008700063860704930444026F0000028327840404
:100880009387F7FF2324F404832784046358F0023A
:10089000832744026384070213850400EF30102B82
:1008A000E30E05FCEF30D057832784049387F7FFCE
:1008B0002324F40483278404E34CF0FC9307F0FF23
:1008C0002324F404EF30D07CEF30507983274404A4
:1008D000635AF00483270401638607049304040128
:1008E0006F000002832744049387F7FF2322F40458
:1008F000832744046358F0028327040163840702BA
:1009000013850400EF309024E30E05FCEF305051C6
:10091000832744049387F7FF2322F40483274404A6
:10092000E34CF0FC9307F0FF2322F404032481003E
:100930008320C10083244100130101016F305075F1
:10094000630A0508130101FE232C8100130405002E
:10095000232E1100232A910023282101232631016F
:1009600013890500EF30906F832404048325C403AA
:100970008329040013850400EF8000051307F0FFAE
:10098000232C0402B3079540B387F9003385A900EF
:100990002322E4042322A400232434012326F40088
:1009A0002324E404631C09028327040163920704DF
:1009B000EF30106E8320C1010324810183244101A3
:1009C000032901018329C10013051000130101024D
:1009D00067800000737004306F000000130504018D
:1009E000EFF0DFD413054402EFF05FD46FF05FFC4B
:1009F00013050401EF30901593071000E31AF5FA80
:100A0000EFF01FB96FF0DFFA631605007370043062
:100A10006F000000130101FE232A91002328210109
:100A200023263101232E1100232C8100930405007D
:100A300013890500930906006380050AEF70D078DA
:100A400013055505EF50804913040500630E050892
:100A5000930745052320F500232E94022320240527
:100A6000EF30D05F832404048325C40303290400EA
:100A700013850400EF7050759306F0FF232C0402D9
:100A8000B30795403307A900B307F9002322D40424
:100A90002322E4002326F4002324D40413050401B4
:100AA00023242401EFF09FC813054402EFF01FC870
:100AB000EF30105E23083405130504008320C101C4
:100AC0000324810183244101032901018329C100F9
:100AD000130101026780000013054005EF5000403C
:100AE0001304050063160500737004306F000000E6
:100AF000232084006FF05FF66316050073700430E6
:100B00006F0000006376B500737004306F00000062
:100B1000130101FF23248100130620001384050024
:100B20009305000023261100EFF01FEE630C050073
:100B3000232C85028320C1000324810013010101BD
:100B400067800000737004306F000000130101FB28
:100B50002326110423248104232291042320210528
:100B6000232E3103232C4103232A5103232861031D
:100B7000232671032326C10063060528638C0526FE
:100B800093072000639CF6000327C503930710001A
:100B90006306F700737004306F00000013890600CD
:100BA0009384050013040500EF30902B631A0500B1
:100BB0008327C10063860700737004306F00000054
:100BC000EF30D049032784038327C403130B0000AD
:100BD000930B20009309F0FF130A0401930A4402C7
:100BE0006364F710630479238327C10063820736A7
:100BF00063160B0013058101EF301010EF305049E0
:100C0000EF20803BEF309045832744046394370105
:100C100023220404832784046394370123240404D7
:100C2000EF3010479305C10013058101EF30D00F5D
:100C300063160530EF309042032784038327C403F3
:100C40006304F710EF30D044EF3050418327840421
:100C50006346F0026F00000313850A00EF30006F57
:100C600063040500EF30D01B832784049387F7FFCC
:100C70002324F404832784046356F000832744026A
:100C8000E39C07FC23243405EF309040EF30103D07
:100C9000832744046346F0026F00000313050A0033
:100CA000EF30C06A63040500EF30901783274404D7
:100CB0009387F7FF2322F404832744046356F0004C
:100CC00083270401E39C07FC23223405EF30503CCA
:100CD000EF200062130B1000EF305038032784031D
:100CE0008327C403E370F7F00326040463040612A9
:100CF000631A091E0325840093850400EF50803E8B
:100D0000832784008326040403274400B387D70085
:100D10002324F40063E4E71083278403832604007C
:100D200003274402938717002324D400232CF402C2
:100D30006300071013054402EF3040619307100071
:100D40006318F50E6F004014EF3090348325C10016
:100D500013050A00EF308032EF30503083278404CF
:100D60006346F0026F00000313850A00EF30005E57
:100D700063040500EF30D00A832784049387F7FFCC
:100D80002324F404832784046356F0008327440259
:100D9000E39C07FC23243405EF30902FEF30102C18
:100DA000832744046346F0026F00000313050A0022
:100DB000EF30C05963040500EF30900683274404E8
:100DC0009387F7FF2322F404832744046356F0003B
:100DD00083270401E39C07FC23223405EF30502BCA
:100DE000EF200051E31805EEEFF08FFA130B10001F
:100DF0006FF09FEE83270504E38407D873700430F7
:100E00006F000000737004306F00000003260404BC
:100E1000631006088327040063860704832784037E
:100E20000327440293871700232CF402E31407F0EE
:100E3000EF301026130510008320C1040324810421
:100E400083244104032901048329C103032A810364
:100E5000832A4103032B0103832BC10213010105E4
:100E60006780000003254400EF305012832784037D
:100E7000032744022322040093871700232CF40243
:100E8000E31A07EAE30605FAEFF08FF06FF05FFA76
:100E90000325C40093850400EF50C0248327040475
:100EA0000327C40083260400B307F0403307F7008C
:100EB0002326E400637ED70403274400B307F7002A
:100EC0002326F40013072000832744026304E90467
:100ED0000327840313071700232CE402E38A07F493
:100EE0006FF05FE50325C40093850400EF50801F79
:100EF000832704040327C40083260400B307F040BB
:100F00003307F7002326E400E37ED7FA6FF0DFFA19
:100F10008327440203278403E30C07FA032784038F
:100F20001307F7FF232CE40203278403130717009A
:100F3000232CE402E38E07EE6FF0DFDF13050400DD
:100F4000EFF0DF90EF20C03A130500006FF0DFEE06
:100F5000EF301014130500006FF01FEE130101FFB6
:100F600023229100930405001305400523248100EA
:100F700023261100EF40907613040500630C05044E
:100F8000232C05029307F0FF2322F504130710001A
:100F900013050501232EE4022324F4042322040074
:100FA0002320040023240400232604002320040417
:100FB00023089404EFF08FF713054402EFF00FF7C6
:100FC00093060000130600009305000013050400BB
:100FD000EFF0DFB7130504008320C1000324810074
:100FE00083244100130101016780000063040504AC
:100FF000130101FF232481002322910023261100E5
:10100000232021010329450013040500EF3040642B
:10101000930400006304A9028320C100032481001B
:1010200013850400032901008324410013010101F9
:1010300067800000737004306F0000008327C400D5
:10104000930410009387F7FF2326F400E39607FC30
:10105000930600001306000093050000130504002A
:10106000EFF0DFAE6FF05FFB130101FC232E1102E6
:10107000232C8102232A91022328210323263103D2
:10108000232441032326C100630E050A93090000AF
:10109000638405101389060093840500130405007A
:1010A000130A05016F008003EF30807EEF30007B74
:1010B0009305C10013058101EF3000476310050659
:1010C000EF30C079032784038327C403630CF7023E
:1010D000EF30007CEF30C07B93091000EF300078D8
:1010E000032784038327C4036362F7068327C100B1
:1010F00063860702E39A09FA13058101EF30C03FC6
:101100006FF09FFAEF30C0788325C10013050A0005
:10111000EF20D076EFF0CFC76FF0DFFBEF304077F6
:101120008320C10303248103832441030329010392
:101130008329C102032A810213050000130101045F
:1011400067800000737004306F0000000326040401
:101150006314060683270400638807048327840337
:101160000327440293871700232CF4026310070817
:10117000EF3000728320C1030324810383244103E1
:10118000032901038329C102032A810213051000E8
:10119000130101046780000083270504E38C07EE38
:1011A000737004306F00000003254400EF30005ED0
:1011B000232204006FF09FFA6316090403258400BC
:1011C00093850400EF401072832784008326040473
:1011D00003274400B387D7002324F400E3E0E7F8B3
:1011E000832704002324F4006FF05FF71305440203
:1011F000EF30C01593071000E31CF5F6EFF04FB980
:101200006FF01FF70325C40093850400EF40906D35
:10121000832704040327C40083260400B307F04097
:101220003307F7002326E4006378D7000327440040
:10123000B307F7002326F40093072000E310F9F228
:1012400083278403E38C07F0832784039387F7FFC6
:10125000232CF4026FF09FF0130101FC232E1102E6
:10126000232C8102232A91022328210323263103E0
:10127000232441032326C1006308051493040000BE
:10128000638C051293890600138905001304050079
:10129000130A45026F000001EF30805FEF30405FBE
:1012A00093041000EF30805B83278403639E07085C
:1012B0008327C100638C070463840404EF30405D1E
:1012C000EF30C0599305C10013058101EF30C025EF
:1012D000631E0502EF30805883278403E39E07FADC
:1012E000EF30005B83270400638607048325C10079
:1012F00013050A00EF209058EFF08FA96FF01FFA46
:1013000013058101EF30401F6FF05FFBEF30405855
:101310008320C103032481038324410303290103A0
:101320008329C102032A810213050000130101046D
:1013300067800000EF30805203254400EF30003515
:10134000EF3000556FF09FFA032604048324C40095
:101350006304060203274400B387C4002326F40075
:1013600063E6E700832704002326F4008325C400F6
:1013700013050900EF401057639C09048327840379
:10138000032704009387F7FF232CF402631607005A
:10139000EF3040572322A400832704016380070411
:1013A00013050401EF20907A930710006318F502EB
:1013B000EFF00F9E6F00800283270504E38407ECA3
:1013C000737004306F000000737004306F00000011
:1013D000832744022326940063960702EF30404B94
:1013E0008320C103032481038324410303290103D0
:1013F0008329C102032A810213051000130101048D
:101400006780000013054402EF205074E30805FCD8
:101410006FF01FFA6302050A63880508130101FED5
:10142000232C8100232A9100232821012324410118
:10143000232E1100232631019307200093840600F8
:1014400013090600138A050013040500639CF600C7
:101450000327C503930710006302F70A7370043073
:101460006F000000EFF00FA7032784038327C40356
:10147000930905006366F7049304000013850900CF
:10148000EFF0CFA48320C101032481011385040060
:1014900003290101832441018329C100032A81001A
:1014A000130101026780000083270504E38807F623
:1014B000737004306F000000737004306F00000020
:1014C00003260404631E060C8327040063860712A8
:1014D000832784031307F0FF93871700232CF4025C
:1014E000832784046388E70E832784049304100011
:1014F000938717002324F4046FF05FF8EFF08F9DBB
:10150000032784038327C403930905006360F70658
:1015100003260404E30A06FA0325C40093050A001F
:10152000EF40503C832704040327C40083260400B3
:10153000B307F0403307F7002326E4006378D700B1
:1015400003274400B307F7002326F4009307200085
:10155000E390F4F883278403E38C07F6832784035E
:101560009387F7FF232CF4026FF09FF60326040401
:10157000E30C06F40325C40093050A00EF409036FF
:10158000832704040327C40083260400B307F04024
:101590003307F7002326E400E364D7FA6FF09FFBDC
:1015A000E39C04F60325840093050A00EF40903382
:1015B000832784008326040403274400B387D700CD
:1015C0002324F400E3E6E7F0832704002324F40057
:1015D0006FF01FF08327440293041000E38007EAB2
:1015E00013054402EF209056E30A05E8E30809E8F2
:1015F000232099006FF09FE803254400EF30001985
:10160000232204006FF0DFEC6302050A8327050440
:1016100063860700737004306F00000083270500A5
:10162000638A0708130101FE232C8100232A9100FD
:10163000130405002328210123263101232E110044
:1016400013890500EFF00F89032784038327C40360
:1016500093090500930400006376F702832784034F
:101660001307F0FF93871700232CF40283278404C9
:10167000638AE70483278404930410009387170088
:101680002324F40413850900EFF04F848320C10163
:1016900003248101138504000329010183244101EE
:1016A0008329C100130101026780000073700430B8
:1016B0006F00000083274500E38607F6737004304F
:1016C0006F00000083274402639607009304100014
:1016D0006FF05FFB13054402EF205047E30805FE5F
:1016E000E30609FE930710002320F9006FF01FFEA8
:1016F000130101FC232E1102232C8102232A9102C3
:1017000023282103232631032324410323225103C9
:101710002326C10063060528638C0526938A0600EC
:101720009389050013040500EF209073631A0500E8
:101730008327C10063860700737004306F000000C8
:10174000EF30C011832784036394071C8327C100F3
:101750006380071013058101EF20105A9304F0FFF6
:1017600013094402130A0401EF308012EF10D00471
:10177000EF30C00E832744046394970023220404AF
:10178000832784046394970023240404EF304010DB
:101790009305C10013058101EF2010596310052442
:1017A000EF30C00B83278403638A070AEF30400EB3
:1017B000EF30C00A832784046346F0026F00000301
:1017C00013050900EF20903863040500EF205065F1
:1017D000832784049387F7FF2324F4048327840456
:1017E0006356F00083274402E39C07FC23249404FF
:1017F000EF30000AEF308006832744046346F0028E
:101800006F00000313050A00EF2050346304050045
:10181000EF201061832744049387F7FF2322F40409
:10182000832744046356F00083270401E39C07FCEC
:1018300023229404EF30C005EF10902BEF3000020C
:10184000832784036396070C8327C100E39E07F078
:10185000EF300004130500006F00800FEF304003ED
:1018600083270400638807108325C100130509003E
:10187000EF20D000EF20907E832784046346F0029F
:101880006F00000313050900EF20502C63040500CE
:10189000EF201059832784049387F7FF2324F4044F
:1018A000832784046356F00083274402E39C07FCEB
:1018B00023249404EF20D07DEF20507A8327440422
:1018C0006346F0026F00000313050A00EF201028A2
:1018D00063040500EF20D054832744049387F7FF67
:1018E0002322F404832744046356F0008327040171
:1018F000E39C07FC23229404EF209079EF10501F03
:1019000063040508EF20907583278403E38E07F2B4
:1019100093850900130504008324C400EFE0DFEF82
:1019200063940A0883278403032704009387F7FF3F
:10193000232CF40263160700EF20D07C2322A4009E
:101940008327040163920708EF20907413051000A9
:101950008320C1030324810383244103032901035A
:101960008329C102032A8102832A4102130101044F
:1019700067800000EF20906E03254400EF20105197
:10198000EF2010716FF05FEEEFE09FC06FF09FF7F8
:1019900083270504E38407D8737004306F000000C8
:1019A000737004306F0000008327440223269400E4
:1019B000E38C07F813054402EF205019E30605F8FD
:1019C000EFE01FBD6FF05FF813050401EF20101862
:1019D00093071000E31AF5F66FF09FFE130504005D
:1019E000EFE0DFE6EF10D010130500006FF05FF6B8
:1019F00063000506130101FF232481002320210138
:101A00002326110023229100832445001389050019
:101A100013040500EF20D0436380A4049306000064
:101A2000130609009305000013050400EFF05FCCD6
:101A300093071000630CF5028320C100032481008A
:101A40008324410003290100130101016780000084
:101A5000737004306F0000008327C400130510006A
:101A6000938717002326F4006FF01FFD8327C4001F
:101A7000938717002326F4006FF01FFC6308050608
:101A80006386050C130101FE232C8100232A91009B
:101A900023282101232631012324410113040500B9
:101AA000232E11001309060093890500EFE09FC261
:101AB00083278403130A050093040000639C070234
:101AC00013050A00EFE09FC08320C10103248101B8
:101AD0001385040003290101832441018329C100E6
:101AE000032A810013010102678000007370043033
:101AF0006F00000003260404630406028325C4006B
:101B000083274400B385C5002326B40063E6F500AF
:101B1000832504002326B40013850900EF40805C70
:101B2000832784031307F0FF9387F7FF232CF40226
:101B3000832744046384E70283274404930410004A
:101B4000938717002322F4046FF09FF7832705047F
:101B5000E38A07F2737004306F00000083270401EA
:101B600063960700930410006FF09FF513050401BE
:101B7000EF20C07DE30805FEE30609FE9307100091
:101B80002320F9006FF01FFE630605088327050474
:101B9000638A050863840708130101FE232C810072
:101BA000232A910023282101232441011304050045
:101BB000232E110023263101138A0500EFE09FB187
:101BC000832784031309050093040000638E070034
:101BD0008329C40093050A0013050400EFE0DFC366
:101BE000930410002326340113050900EFE01FAE13
:101BF0008320C1010324810113850400032901010D
:101C0000832441018329C100032A810013010102B9
:101C100067800000737004306F0000007370043040
:101C20006F000000E38C07FE737004306F0000004B
:101C300063160500737004306F000000130101FF8C
:101C4000232481001304050023261100EF201041F6
:101C500003248403EF20D0438320C1001305040034
:101C60000324810013010101678000006316050051
:101C7000737004306F000000130101FF2326110070
:101C80002324810013040500EF20503D83278403A3
:101C90000324C4033304F440EF20903F13050400F1
:101CA0008320C1000324810013010101678000002B
:101CB0006306050003258503678000007370043008
:101CC0006F0000006308050497870300938787AFC0
:101CD00003A747006304E50403A7C7006302E50800
:101CE00003A74701630AE50603A7C7016302E506E8
:101CF00003A74702630AE50403A7C7026302E504DA
:101D000003A74703630AE50203A7C7036302E502CB
:101D10006F40C034737004306F0000001307000080
:101D200013173700B387E70023A007006F40003385
:101D3000130770006FF0DFFE130760006FF05FFEA7
:101D4000130750006FF0DFFD130740006FF05FFDD9
:101D5000130730006FF0DFFC130720006FF05FFC0B
:101D6000130710006FF0DFFB0325C5046780000038
:101D70002326B50467800000034505056780000041
:101D800063080500032585031335150067800000EF
:101D9000737004306F000000630C05008327850317
:101DA0000325C5033305F540133515006780000092
:101DB000737004306F00000097870300938787A03B
:101DC00003A707006300070403A78700630807044D
:101DD00003A707016308070403A787016308070433
:101DE00003A707026308070403A787026308070421
:101DF00003A70703630C070403A78703630407040F
:101E0000678000001307000013173700B387E7004F
:101E100023A0B70023A2A7006780000013071000CB
:101E20006FF09FFE130720006FF01FFE13073000B6
:101E30006FF09FFD130740006FF01FFD1307500068
:101E40006FF09FFC130770006FF01FFC130760001A
:101E50006FF09FFB978703009387C79603A7470000
:101E60006300E50403A7C7006306E50403A7470171
:101E70006306E50403A7C7016306E50403A7470259
:101E80006306E50403A7C7026306E50403A7470347
:101E9000630AE50403A7C7036302A7046780000081
:101EA0001307000013173700B387E70023A00700CC
:101EB00067800000130710006FF0DFFE130720009B
:101EC0006FF05FFE130730006FF0DFFD1307400077
:101ED0006FF05FFD130750006FF0DFFC1307700019
:101EE0006FF05FFC130760006FF0DFFB130101FF71
:101EF00023248100232291002320210113040500C3
:101F0000232611009384050013090600EF20101505
:101F1000032744049307F0FF6314F700232204040B
:101F2000032784049307F0FF6314F70023240404B9
:101F3000EF20101683278403639A07001306090015
:101F40009385040013054402EF20802FEF20101129
:101F500083278404635AF0048327440263860704BA
:101F6000930444026F000002832784049387F7FFE1
:101F70002324F404832784046358F0028327440253
:101F80006384070213850400EF20403CE30E05FC48
:101F9000EF200069832784049387F7FF2324F40448
:101FA00083278404E34CF0FC9307F0FF2324F4041C
:101FB000EF20100EEF20900A83274404635AF004A8
:101FC0008327040163860704930404016F00000261
:101FD000832744049387F7FF2322F40483274404D0
:101FE0006358F00283270401638407021385040009
:101FF000EF20C035E30E05FCEF2080628327440408
:102000009387F7FF2322F40483274404E34CF0FC76
:102010009307F0FF2322F404032481008320C100EE
:102020008324410003290100130101016F205006A0
:1020300097E701009387875483A6070017E70100FD
:10204000130787520327070023A2A600636AE5044B
:10205000130101FF232481002326110017E701004B
:1020600013078751130405000325070083A5070004
:1020700093854500EFE00FF197E701009387074D47
:1020800083A707006376F40097E7010023A0874C3D
:102090008320C10003248100130101016780000037
:1020A00017E701001307074D0325070083A5070065
:1020B000938545006FE00FED97E701009387074C8C
:1020C00003A7070083A60700832747049387F7FF2A
:1020D0002322F70483A74604639407007360043047
:1020E0006780000063020504130101FD232E310106
:1020F000232A510123261102938A070023248102F7
:102100002322910223202103232C41012328610152
:1021100023267101930740009309070063FAE70043
:10212000737004306F000000737004306F000000A3
:10213000130B05009384050013090600938B06001A
:10214000130A08006302082C13050006EF3010592B
:10215000130405006302052A1319290023284503E7
:10216000130609009305500A13050A00EF40800981
:1021700003C70400832704031309C9FF230AE402E9
:1021800003C70400338927011379C9FF6306070ECB
:1021900083C71400A30AF40283C71400638E070CDC
:1021A00083C72400230BF40283C724006386070C33
:1021B00083C73400A30BF40283C73400638E070A7D
:1021C00083C74400230CF40283C744006386070AD4
:1021D00083C75400A30CF40283C75400638E07081E
:1021E00083C76400230DF40283C764006386070875
:1021F00083C77400A30DF40283C77400638E0706BF
:1022000083C78400230EF40283C784006386070615
:1022100083C79400A30EF40283C79400638E07045F
:1022200083C7A400230FF40283C7A40063860704B6
:1022300083C7B400A30FF40283C7B400638E070200
:1022400083C7C4002300F40483C7C4006386070265
:1022500083C7D400A300F40483C7D400638E0700AF
:1022600083C7E4002301F40483C7E4006386070006
:1022700083C7F400A301F404130A440013050A0001
:10228000A30104042326340323283405232A040449
:10229000EFE0CFCB13058401EFE04FCB9307500065
:1022A000B3873741232C040423288400232CF40013
:1022B0002322840223220404232E040413860B0009
:1022C00093050B0013050900EFE08FC12320A40044
:1022D00063840A0023A08A007370043017E90100A8
:1022E000130909288327090097E40100938404292E
:1022F000638C070003A7040083A704008327470417
:10230000938717002322F70417E701001307072616
:10231000832707009387170097E6010023A8F62478
:1023200083A70400638E070E83270900639C0700C0
:1023300083A7040083A7C70263E6F90097E70100BB
:1023400023AE872297E701009387872083A70700A2
:1023500017E70100130707210325C402032707001D
:102360009387170097E6010023A4F61E2324F404A4
:102370006376A70097E7010023A6A71E93054001F7
:10238000EF60806497E701009387872F3385A7006C
:1023900093050A00EFE00FBC83270900638807005C
:1023A00083A7040083A747046390071283270900CB
:1023B00013041000638A070083A7040083A7C702E1
:1023C00063F43701EFE0CF9C130504008320C102C2
:1023D0000324810283244102032901028329C101CC
:1023E000032A8101832A4101032B0101832BC100B0
:1023F000130101036780000013050A00EF30104647
:102400001304F0FF6FF05FFC13152600EF30102D62
:10241000130A0500E31A05D21304F0FF6FF0DFFA88
:1024200097E7010023AC87140327070093071000E8
:10243000E31AF7F017E5010013058524EFE00FAF6D
:1024400017E5010013050525EFE04FAE17E5010084
:1024500013058525EFE08FAD17E50100130505266F
:10246000EFE0CFAC17E5010013058526EFE00FACD8
:1024700017EB0100130B0B2713050B00EFE00FAB5D
:1024800097EA0100938A4A2713850A00EFE00FAA12
:1024900017E5010013058527EFE04FA917E50100B7
:1024A00013050528EFE08FA817E50100130585281F
:1024B000EFE0CFA797E7010023A0670D97E70100A2
:1024C00023AA570B6FF01FE803A7040083A604009C
:1024D000832747049387F7FF2322F70483A7460443
:1024E000E39607EC736004306FF05FEC130101FFBB
:1024F000232481002326110023229100232021017F
:10250000130405007370043097E4010093844405BC
:1025100083A70400639E07106318040097E7010077
:102520009387C70503A40700130944001305090096
:10253000EFE08FAA832784026386070013058401D6
:10254000EFE08FA99305090017E501001305451D6C
:10255000EFE04FA097E701009387870103A70700EB
:1025600097E701009387C7FE83A7070013071700AB
:1025700097E6010023AEE6FE03A704009387170049
:1025800097E6010023A6F6FC630C070097E701001D
:102590009387C7FE03A7070003274704631C070EA2
:1025A00083A70400638A070697E70100938707FD66
:1025B00003A70700630287107370043003A70400A9
:1025C0006318070817E70100130707FB83260700B6
:1025D00083A606006392060A1307F0FF97E6010040
:1025E00023A6E6F603A704006308070203A7070073
:1025F000032747046302070203A7070083A6070017
:10260000832747049387F7FF2322F70483A7460411
:1026100063940700736004308320C10003248100A9
:102620008324410003290100130101016780000098
:1026300097E70100938787F403A7070083A70700A4
:1026400083274704938717002322F7046FF0DFECFA
:1026500083A6070003A7070003A746041307170074
:1026600023A2E60417E70100130707F183260700FA
:1026700083A60600E38206F6032707000327C700A8
:102680000327C7000327470097E6010023A0E6ECD5
:102690006FF05FF503A7070083A6070083274704B1
:1026A0009387F7FF2322F70483A74604E39A07EEF4
:1026B000736004306FF0DFEE97E701009387C7E89F
:1026C00083A7070063860700737004306F00000063
:1026D000032481008320C1008324410003290100D9
:1026E000130101016FD0DFEA6304050C17E7010055
:1026F0001307C7E883260700930700006386A60A2E
:10270000130101FF232611002324810023229100BD
:102710007370043097E60100938686E483A7060071
:10272000638C0700032607008327070083274604DE
:10273000938717002322F60483A70600930405005D
:1027400003244501638807008327070083A7470404
:102750006394070697E70100938707E283A70700C2
:10276000638C870697E701009387C7E083A707007C
:102770006384870697E701009387C7FB6306F40429
:1027800097E701009387C7F9630CF40293071000E1
:102790008320C100032481008324410013850700A6
:1027A00013010101678000001385070067800000A6
:1027B000737004306F000000EFF01F906FF09FF90E
:1027C000930740006FF0DFFC83A7840293B71700E4
:1027D000938727006FF0DFFB930720006FF05FFB0C
:1027E0007370043097E70100938787D703A707002A
:1027F000631607026304050483A707000325C502C7
:10280000638C070097E70100938747D703A707006A
:1028100003274704631C07026780000017E70100D5
:102820001307C7D5832607000327070003A746041D
:102830001307170023A2E604E31005FC17E70100C5
:102840001307C7D3032507006FF01FFB03A707007B
:1028500083A60700832747049387F7FF2322F70403
:1028600083A74604E39A07FA736004306780000088
:10287000130101FF23248100130405002326110006
:10288000EFD05FE56318040097E70100938707CF57
:1028900003A407000324C402EFD05FE38320C10038
:1028A0001305040003248100130101016780000067
:1028B0009307400063F6B700737004306F000000A8
:1028C000130101FE232C8100232E1100232A9100E5
:1028D000232821012326310123244101130405006B
:1028E0007370043017E90100130989C783270900B1
:1028F000639207106300041283270405638EF50AB0
:1029000017E70100130787C763F0B70283260700A4
:10291000638E8612032707008324C702B3B4950091
:1029200093C414006F00000183240700B384844023
:1029300093B414000327C4026386E70E832784013F
:102940002328B40463C8070093075000B385B74039
:10295000232CB40093172700B387E7000327440113
:1029600097E901009389C9D193972700B387F900AC
:102970006310F704130A440013050A00EFD0DFE5E3
:1029800097E70100938707BE0325C40283A70700CA
:1029900063F6A70097E7010023A6A7BC93054001B3
:1029A000EF60800293050A003385A900EFD09FDA1B
:1029B00063840400EFD0DFBD83270900638C070028
:1029C00097E70100938787BB83A7070083A7470486
:1029D000639E07048320C1010324810183244101F4
:1029E000032901018329C100032A81001301010287
:1029F0006780000097E70100938747B803A70700A7
:102A000083A7070083274704938717002322F7042F
:102A1000E31404EE97E70100938747B603A4070089
:102A20006FF09FED2326B4026FF05FF10324810164
:102A30008320C10183244101032901018329C100AD
:102A4000032A8100130101026FF00FE793040000D5
:102A50006FF05FEE630A0508130101FE232A91005F
:102A600097E40100938484B183A70400232E11000E
:102A7000232C810023282101232631016388A70408
:102A80007370043017E90100130989AD8327090029
:102A9000638C070003A7040083A70400832747046F
:102AA000938717002322F7040327450197E70100C6
:102AB000938747C8630EF7028327090063880700DE
:102AC00083A7040083A74704639E07088320C101EE
:102AD0000324810183244101032901018329C100C9
:102AE0001301010267800000737004306F00000062
:102AF0008327850217E70100130747C1E38EE7FA32
:102B0000E39C07FA930945001304050013850900A7
:102B1000EFD09FCC97E701009387C7A40325C40299
:102B200083A7070063F6A70097E7010023ACA7A2DD
:102B300093054001EF50506997E70100938747B430
:102B40003385A70093850900EFD0DFC083A7040079
:102B50000327C40283A7C702E360F7F6EFD05FA3A1
:102B60006FF09FF5032481018320C101832441017B
:102B7000032901018329C100130101026FF0CFD3A2
:102B800063020506130101FE232C8100232A910014
:102B90002326310113040500232E110023282101CF
:102BA000EFD05FB30327440197E70100938787B80D
:102BB0009309050093040000630AF70213850900D6
:102BC000EFD0DFB08320C10103248101138504000D
:102BD00003290101832441018329C100130101025A
:102BE00067800000737004306F0000008327840248
:102BF00017E50100130585B1E382A7FCE39007FC0C
:102C000097E701009387479483A70700639407061B
:102C100097E701009387879683A707008324C40260
:102C20001309440083A7C70213050900B3B4F400D5
:102C3000EFD09FBA97E701009387C7920325C4029C
:102C400083A7070093C4140063F6A70097E7010069
:102C500023AAA79093054001EF50105797E7010072
:102C6000938707A2930509003385A700EFD09FAE95
:102C70006FF0DFF493058401EFD0DFAD6FF01FF448
:102C8000130101FE37150000232E1100232C8100B3
:102C9000232A9100232821012326310123244101E5
:102CA00023225101EF30802363060524930405009D
:102CB00013050006EF308022130405006300052889
:102CC000371600009305500A232895021385040047
:102CD000EF30405383240403B71700009387C7FFE6
:102CE000B384F400B7474C45938797449309440055
:102CF000232AF40213850900230C0402A30104040F
:102D00002326040223280404232A0404EFD01FA44A
:102D100013058401EFD09FA393075000232C0404D4
:102D200093F4C4FF23288400232CF400232284027C
:102D300023220404232E0404130600009715000028
:102D4000938585EA13850400EFD09F992320A40082
:102D50007370043017E90100130989808327090083
:102D600097E4010093848481638C070003A7040027
:102D700083A7040083274704938717002322F704BF
:102D800017D701001307877E832707009387170053
:102D900097D6010023ACF67C83A704006388070A5A
:102DA00083270900639C070083A7040083A7C70249
:102DB0006396070097D7010023A2877C97D701006D
:102DC0009387077983A7070097D6010093868679B2
:102DD0000327C40283A606009387170017D60100B5
:102DE0002328F6762324F40463F6E60097D701003F
:102DF00023AAE77693172700B387E7009397270066
:102E000017E501001305C5873305F5009385090013
:102E1000EFD05F94832709006388070083A704002D
:102E200083A74704639A070E83270900638407007A
:102E300083A70400EF201007930710006304F51226
:102E4000631A050A737004306F00000097D7010001
:102E500023A687720327070093071000E310F7F6F5
:102E600017E501001305C581EFD05F8C17E5010060
:102E700013054582EFD09F8B17E501001305C5822E
:102E8000EFD0DF8A17E5010013054583EFD01F8AD5
:102E900017E501001305C583EFD05F8997EA0100AC
:102EA000938A4A8413850A00EFD05F8817EA0100ED
:102EB000130A8A8413050A00EFD05F8717E5010023
:102EC0001305C584EFD09F8617E5010013054585DE
:102ED000EFD0DF8517E501001305C585EFD01F850D
:102EE00097D7010023AA576997D7010023A4476900
:102EF0006FF0DFEC8320C1010324810183244101B1
:102F0000032901018329C100032A8100832A41008A
:102F1000130101026780000003A7040083A60400D8
:102F2000832747049387F7FF2322F70483A74604E8
:102F3000E39C07EE736004306FF01FEF0324810100
:102F40008320C101032901018329C100032A8100D3
:102F5000832A4100138504008324410113010102E7
:102F60006F30C00F737004309307F0FF17D7010064
:102F7000232EF75C0324810197D7010023A2A75ECB
:102F80008320C10183244101032901018329C10058
:102F9000032A8100832A410097D7010023A6075CFA
:102FA000130101026FD00FC47370043097D7010072
:102FB00023A8075A6FD04FD517D701001307C7585A
:102FC00083270700938717002320F70067800000FE
:102FD0007370043097D701009387875803A70700C1
:102FE0006318070217D701001307075803250700C6
:102FF00083A70700638C070097D7010093870758C2
:1030000003A7070003274704631407026780000033
:1030100017D70100130787568326070003270700E9
:1030200003A746041307170023A2E6046FF09FFBD3
:1030300003A7070083A60700832747049387F7FFAA
:103040002322F70483A74604E39207FC736004304D
:1030500067800000130101FF232611002324810053
:10306000EFD04FE797D701009387075003A40700DD
:10307000EFD0CFE58320C1001305040003248100B5
:10308000130101016780000097D701009387074E65
:1030900003A5070067800000130101FD232611022C
:1030A000232481022322910223202103232E310194
:1030B000232C4101232A5101232861012326710178
:1030C00097D701009387474883A70700639A0706AD
:1030D00017D7010013074749832707009387170075
:1030E00097D6010023A2F648832A0700638A0A0ABA
:1030F00097D701009387874583A7070093040000B3
:1031000063FEFA0A97D901009389895717DA0100FB
:10311000130ACA4683270A009306100003A7C702B2
:1031200093172700B387E70093972700B389F90027
:1031300083A7090063F4F602930410006F000002F5
:1031400097D701009387874183A707009304000066
:103150009387170017D701002322F74097D7010064
:103160009387873F83A707006384070093041000B9
:103170008320C10203248102138504000329010274
:10318000832441028329C101032A8101832A410149
:10319000032B0101832BC100130101036780000091
:1031A00017D401001304443D8327040083A70700BC
:1031B0006388070C737004306F00000017D401009F
:1031C0001304843B97D901009389894B17DA0100D6
:1031D000130ACA3A17DB0100130BCB38832704000C
:1031E00083A70700638007088327040083A7C7001D
:1031F00003A9C70083274900930B490013850B00DF
:1032000063EAFA06EFD04FDD8327890213058901AF
:1032100063840700EFD04FDC8327C90203270B002C
:1032200093850B00139527003305F5001315250032
:103230003385A9006376F70017D701002324F732FE
:10324000EFD04FD183270A000327C90283A7C70203
:10325000E366F7F8832704009304100083A70700B0
:10326000E39407F89307F0FF17D701002320F72E08
:103270006FF05FEA17D70100232AF72C6FF09FE960
:1032800017D701001307072F832704000327070020
:1032900097D6010023A2E62E17D70100232CF72C86
:1032A00097D701009387072B83A707009387170001
:1032B00017D701002320F72A8327040083A70700DC
:1032C000639A07009307F0FF17D701002320F72820
:1032D0006FF01FE28327040083A7C70083A7C700FE
:1032E00083A7470017D701002322F7266FF05FE07E
:1032F00097D701009387472503A7070063160700A8
:10330000737004306F000000130101FE232E1100C2
:10331000232C8100232A9100232821012326310117
:1033200023244101232251012320610173700430C1
:1033300097D401009384C42203A7040063100712EA
:1033400003A707001307F7FF97D6010023AEE61E79
:1033500083A70700639E070A97D701009387072179
:1033600083A707006386070A97DA0100938A4A3128
:1033700017DA0100130A0A1F17D9010013090920DF
:10338000930910006F00C0013385EA00EFD08FBCB5
:10339000832709000327C40283A7C7026374F706C3
:1033A00083A7CA086380070E83A78A0903A4C700FE
:1033B00013058401EFD04FC2130B440013050B001B
:1033C000EFD08FC18327C40283260A0093050B0028
:1033D000139527003305F500131525001307050085
:1033E0003385AA00E3F2F6FA17D70100232CF7166B
:1033F000EFD04FB6832709000327C40283A7C70273
:10340000E360F7FA97D7010023A837156FF05FF94B
:103410001304000083A70400638C070097D7010002
:103420009387C71583A7070083A7470463980704FA
:10343000130504008320C101032481018324410179
:10344000032901018329C100032A8100832A410045
:10345000032B0100130101026780000017D7010050
:103460001307C711832607000327070003A7460495
:103470001307170023A2E6046FF09FECEFE0DFC311
:103480006FF01FFB17D401001304440D83270400C1
:10349000638C070283270400130910006386070268
:1034A000EFF09FBF6306050097D7010023A6270B07
:1034B000832704009387F7FF17D701002320F70A1B
:1034C00083270400E39E07FC97D701009387C70872
:1034D00003A7070093071000E31CF7F2EFD04F8B10
:1034E000130410006FF01FF36304050263960500D8
:1034F000737004306F00000017D701001307C70472
:1035000083270700638A0700737004306F00000090
:10351000737004306F000000130101FF2324810049
:103520002326110083260700032705009386160033
:1035300017D60100232AD60097D601009386C6022B
:1035400083A606003304B7002320850063F0E60459
:103550006372E40263F0860297D701009387070243
:1035600003A5070013054500EFD00FA713050400BE
:10357000EFE01FACEFF0DFD7630E05008320C10042
:10358000032481001301010167800000E366E4FC6D
:103590006FF05FFC032481008320C100130101014F
:1035A0006FC01FFF630E050017D701001307C7F98F
:1035B0008327070063880700737004306F000000E2
:1035C0006FC01FFD130101FF23261100232481007A
:1035D00003270700930705001307170097D601007C
:1035E00023A4E6F697D60100938646F917D7010083
:1035F000130787F70327070003A506003304F70026
:1036000013054500EFD04F9D13050400EFE05FA2C6
:10361000EFF01FCE631A0500032481008320C10050
:10362000130101016FC0DFF68320C1000324810074
:103630001301010167800000130101FF23248100B1
:103640002326110097D70100938707F083A707006F
:10365000130400009387170017D701002326F7EE05
:1036600097D70100938787F083A7070063ECF50ED7
:1036700017DE0100130E4E0697D20100938282FFDF
:103680001304000013070000930F10001303500AE7
:103690006F00C000130ECEFE6386C21183278EFF1B
:1036A00093050700E38807FE8327CEFF83A7470023
:1036B000232EFEFE6388C72103AFC70083A7470000
:1036C0003307E500930E0000232EFEFE6380C7093A
:1036D00083A8C70093874803232017012322F700FC
:1036E00083A788042326F7012324F70083A7C802B1
:1036F0002328F70083A70805232C0700232AF700B7
:1037000003A8080383470800639A67069307080025
:103710009387170083C60700B3850741E38A66FED7
:1037200093D525009395050193D50501231EB70078
:10373000938E1E0013070702630C1F058327CEFF1D
:1037400083A74700232EFEFEE394C7F983274E008C
:10375000232EFEFE6FF0DFF73304640063040600DF
:1037600023200600EFF0DFB8130504008320C1001A
:10377000032481001301010167800000930500000C
:10378000231EB700938E1E0013070702E3181FFBCA
:103790003304D40113175400130ECEFE9305070013
:1037A000E39EC2EF97D70100938707DD03AE0700C2
:1037B00083270E00639E071097D70100938787DB4E
:1037C00003AE070083270E006392071C17DE01007B
:1037D000130E0EEB83270E0A6398072683274E0BE2
:1037E000E38E07F683278E0B97DE0100938E0EF58E
:1037F00083A7470017D701002320F7F4638CD73D38
:1038000083AFC70083A747003307B5001303000049
:1038100097D6010023A2F6F2130F30009302200086
:103820009308500A6388D70903A5C7009307450387
:103830002320A7002322F700832785042326E701FE
:103840002324F7008327C5022328F7008327850256
:10385000638407002326570083270505232C0700D0
:10386000232AF7000328050383470800639C1733C6
:10387000930708009387170083C60700B3850741A5
:10388000E38A16FF93D525009395050193D505018D
:10389000231EB7001303130013070702E38EAFEADA
:1038A00083278E0B83A7470097D6010023A6F6E84F
:1038B000E39CD7F783270E0C97D6010023AEF6E6DC
:1038C0006FF09FF683274E00232EFEFE6FF0DFDEA3
:1038D00083274E00130F8E0083A647002322DE00AD
:1038E000638CE62DB307E50003A7460083A2C6005C
:1038F000930E00002322EE00930F20001303500AC2
:103900006300EF088328C7001387480323A017012B
:1039100023A2E70003A7880423A6F70123A4E70056
:1039200003A7C80223A8E70003A7080523AC0700E4
:1039300023AAE70003A8080303470800631A6722C5
:10394000130708001307170083460700B305074154
:10395000E38A66FE93D525009395050193D505016D
:10396000239EB700938E1E0093870702638C12215B
:1039700083264E0003A746002322EE00E314EFF84F
:103980000327CE002322EE006FF0DFF783274E00DF
:10399000130F8E0083A747002322FE006388E721D0
:1039A00083A2C70083A74700B305B500930E0000AC
:1039B0002322FE00930F20001303500A6300FF0828
:1039C00083A8C7009387480323A0150123A2F5000D
:1039D00083A7880423A6F50123A4F50083A7C802C2
:1039E00023A8F50083A7080523AC050023AAF5004A
:1039F00003A808038347080063946714930708002B
:103A00009387170083C6070033870741E38A66FE62
:103A1000135727001317070113570701239EE500CB
:103A2000938E1E00938505026386121383274E0032
:103A300083A747002322FE00E314FFF88327CE006C
:103A40002322FE006FF0DFF783274E0A17DF010005
:103A5000130F8FCD83A7470017D701002324F7CC7E
:103A60006382E71783A2C70083A74700B305B500A9
:103A7000930E000017D701002326F7CA930F4000CA
:103A80001303500A6382E70983A8C700938748039A
:103A900023A0150123A2F50083A7880423A6F5011E
:103AA00023A4F50083A7C80223A8F50083A708056F
:103AB00023AC050023AAF50003A8080383470800E8
:103AC000639C6704930708009387170083C6070069
:103AD00033870741E38A66FE135727001317070150
:103AE00013570701239EE500938E1E009385050260
:103AF000638E120383274E0A83A7470017D701005E
:103B00002322F7C2E392E7F98327CE0A17D70100F1
:103B1000232AF7C06FF05FF713070000239EE5002C
:103B2000938E1E0093850502E39612FD83274E0BAC
:103B30003304D40193155400E38207C26FF09FCA87
:103B400013070000239EE500938E1E009385050257
:103B5000E39E12ED17DE0100130E8EB283270E0ACC
:103B60003304D40193155400E38A07C66FF0DFEDE8
:103B700093050000239EB700938E1E0093870702D3
:103B8000E39812DF97D701009387C79E03AE070023
:103B90003304D4019315540083270E00E38807C231
:103BA0006FF0DFDE930500006FF09FCE8327CE001D
:103BB0002322FE006FF0DFDE8326CE002322DE000C
:103BC0006FF05FD28327CE0A17D70100232CF7B4FA
:103BD0006FF05FE983270E0C17D70100232EF7B48F
:103BE0006FF01FC2130101FD232291022320210344
:103BF000232E3101232C4101232A51012328610165
:103C000023267101232611022324810297D9010062
:103C10009389899317D90100130989A617DA01003E
:103C2000130A0A9497DA0100938A4A9597DB0100F8
:103C3000938BCB9397D4010093848493130B100040
:103C40006F00000283A709000324090A9387170065
:103C500017D70100232AF78EEFF08FE9631E0400C7
:103C600083A70400E39007FE83270900E37AFBFEA5
:103C7000EFC01F926FF0DFFE7370043083270A00DD
:103C8000639E07048327C90A03A4C70013054400E1
:103C9000EFC09FB483A70B009387F7FF17D70100EE
:103CA0002326F78C83A704009387F7FF17D701001B
:103CB0002320F78C83270A006388070083A70A0064
:103CC00083A747046398070203250403EF20003904
:103CD00013050400EF2080386FF09FF803A70A0057
:103CE00083A70A0083274704938717002322F7043A
:103CF0006FF05FF903A70A0083A60A008327470431
:103D00009387F7FF2322F70483A74604E39E07FA6D
:103D1000736004306FF05FFB97D701009387C78211
:103D200083A70700639E070E130101FF23261100DE
:103D3000232481002322910097D7010023AE07801E
:103D400017D701001307878383270700B7A6A5A508
:103D50009386565A83A7070383A50700639ED50061
:103D600003A64700631AB60083A687006396C600C1
:103D700083A7C700638AD7000325070083250700B0
:103D800093854503EF30C07617C701001307877D81
:103D90008326070017D401001304848E6F000002ED
:103DA0008327070063860708832707009387F7FFA9
:103DB00097C6010023A8F67A83260700939726006A
:103DC000B387D70093972700B307F40083A70700B2
:103DD000E38807FC0325070093172500B387A70096
:103DE000939727003307F4008326470093878700C3
:103DF000B307F40083A4460023229700638EF402E5
:103E000083A7C4008320C1000324810017C70100D9
:103E10002326F77683244100130101016780000007
:103E20009307100017C701002328F772678000006E
:103E3000737004306F00000083A4440093054001B8
:103E4000EF4090383305A400232295006FF05FFB0C
:103E5000130101FE23282101232E1100232C8100B0
:103E6000232A9100232631011309050073700430C1
:103E700097C401009384C46E83A7040017C4010093
:103E80001304C46F639C070C631409000329040026
:103E90009309490013850900EFC01F948327890205
:103EA0006386070013058901EFC01F9393850900FE
:103EB00017D5010013050588EFC0DF8983A704002B
:103EC000638807008327040083A747046394070AD5
:103ED000832704006384270D83A7040063820706F9
:103EE0007370043083A704006398070E97C701001E
:103EF0009387876803A70700032707006310070C51
:103F00009307F0FF17C701002322F76483A704007B
:103F1000638807028327040083A74704638207029C
:103F20000327040083260400832747049387F7FFB1
:103F30002322F70483A746046394070073600430C8
:103F40008320C1010324810183244101032901014C
:103F50008329C100130101026780000003270400C8
:103F60008327040083274704938717002322F7043D
:103F70006FF09FF103270400832604008327470482
:103F80009387F7FF2322F70483A74604E39207F4FD
:103F90007360043083270400E39027F583A70400AF
:103FA0006382070697C701009387075A83A7070014
:103FB0006388070A737004306F00000083A707004E
:103FC00083A7C70083A7C70083A7470017C70100BF
:103FD000232EF7566FF09FF3032704008327040076
:103FE00083274704938717002322F70497C701000C
:103FF0009387875803A7070003270700E30207F00A
:104000006FF0DFFB97C701009387475617C7010082
:104010001307076783A707000327470B6314F702FB
:104020008320C1010324810197C7010023A80754FD
:1040300083244101032901018329C10013010102E5
:1040400067800000032481018320C1018324410192
:10405000032901018329C100130101026FF0DFCBA5
:10406000032481018320C10183244101032901012B
:104070008329C100130101026FC08FD16306050AB5
:10408000130101FF2322910097C401009384044F80
:10409000232021011389050083A504002326110094
:1040A0002324810093858501EFC0CFED03A5040093
:1040B00013054500EFC04FF29307F0FF630AF906BE
:1040C00097C701009387474A03A4070003A704008A
:1040D00083A707003304240123228700636EF406BC
:1040E00097C701009387474903A5070083A50400EC
:1040F00093854500EFC00FE997C7010093870745F7
:1041000083A707006376F40097C7010023A08744C4
:104110008320C1000324810083244100032901007E
:104120001301010167800000737004306F0000000C
:1041300083A50400032481008320C100832441005F
:104140000329010017C501001305C55E93854500CD
:10415000130101016FC00FE097C7010093878741EA
:1041600003A507000324810083A504008320C10068
:1041700083244100032901009385450013010101B7
:104180006FC04FE0630E050097C701009387C73BE0
:1041900083A70700639A0700737004306F00000064
:1041A000737004306F000000130101FF232291009F
:1041B00097C401009384843C03A7040093870500FF
:1041C00083A50400B7060080B3E7D70023261100BB
:1041D00023248100232CF700938585011304060016
:1041E000EFC04FD703A5040013054500EFC0CFDE95
:1041F0009307F0FF6304F40297C701009387C73663
:1042000003A507008320C1008324410033058500F6
:1042100003248100130101016FD09FE183A50400F5
:10422000032481008320C1008324410017C50100BD
:104230001305455093854500130101016FC08FD1CF
:104240006308050A130101FF2322910097C40100AE
:104250009384C432232021011389050083A504001F
:104260002326110023248100938585011304060071
:10427000EFC04FCE03A5040013054500EFC0CFD516
:1042800093071000630AF40697C701009387C72DB0
:1042900003A4070003A7040083A707003304240135
:1042A00023228700636EF40697C701009387C72C0B
:1042B00003A5070083A5040093854500EFC08FCCBC
:1042C00097C701009387872883A707006376F400C8
:1042D00097C7010023AC87268320C10003248100F7
:1042E00083244100032901001301010167800000BC
:1042F000737004306F00000083A504000324810064
:104300008320C100832441000329010017C5010057
:104310001305454293854500130101016FC08FC30A
:1043200097C701009387072503A507000324810091
:1043300083A504008320C1008324410003290100D8
:1043400093854500130101016FC0CFC3130101FF25
:104350002326110023248100232291008327C500F6
:1043600003A4C7006304040A9304840113850400B2
:10437000EFC08FC697C701009387071D83A707006B
:10438000639A07089304440013850400EFC0CFC468
:1043900097C701009387071D0327C40283A707005F
:1043A00063F6E70097C7010023AEE71A93172700CB
:1043B000B387E7009397270017C501001305452C25
:1043C000938504003305F500EFC0CFB897C701000F
:1043D0009387C71A83A707000327C40213050000A9
:1043E00083A7C70263FAE7009307100017C701000D
:1043F0002324F716130510008320C1000324810035
:1044000083244100130101016780000073700430B0
:104410006F0000009385040017C501001305052FE8
:10442000EFC04FB36FF09FFA97C701009387C71192
:1044300083A7070063960700737004306F000000C5
:10444000130101FF23261100232481002322910060
:10445000B70700800324C500B3E7F5002320F5006B
:1044600063080408EFC04FB79304440013850400A9
:10447000EFC08FB697C701009387C70E0327C4020A
:1044800083A7070063F6E70097C7010023ACE70C9A
:1044900093172700B387E7009397270017C50100FC
:1044A0001305051E3305F50093850400EFC08FAAA0
:1044B00097C701009387870C83A707000327C402CF
:1044C0001305000083A7C70263FAE70093071000F3
:1044D00017C701002322F708130510008320C1002D
:1044E000032481008324410013010101678000003F
:1044F000737004306F0000006304050297C7010069
:104500009387470503A7070097C701009387C7054F
:1045100083A707002320E5002322F5006780000021
:10452000737004306F0000006304050E638E050C89
:10453000130101FF23261100232481001307050026
:104540007370043097C801009388880183A708001E
:104550006380070297C701009387470283A607007D
:1045600083A7070083A746049387170023A2F604B6
:1045700017C30100130343FF83A7050003260300AD
:104580009306F0FF130400006388D70417CE0100E0
:10459000130E4EFC03250E00032807008326470058
:1045A0006306A800130410006378D6023308D640CF
:1045B000130410006372F80203250E00B387C7408E
:1045C00003260300B387D70023A0F5002320A7000C
:1045D0002322C7001304000083A70800638C070090
:1045E00097C70100938787F983A7070083A747042C
:1045F00063940702130504008320C1000324810093
:104600001301010167800000737004306F00000027
:10461000737004306F000000EFD01FAA6FF09FFD91
:104620009307100017C701002328F7F267800000E6
:10463000630605000325C50467800000130500001C
:1046400067800000630405002326B504678000002E
:1046500097C70100938787F203A5070067800000D2
:1046600097C701009387C7EF83A7070013051000C2
:10467000638C070097C70100938707ED03A5070028
:10468000133515001315150067800000630C05082D
:10469000130101FE232A910097C40100938404EEC4
:1046A00083A70400232E1100232C8100232821013D
:1046B000232631010327C50283A7C7026376F704C7
:1046C0008327850163CC070083A7040083A6C70264
:1046D00093075000B387D740232CF500931727008A
:1046E000B387E7000327450117C90100130949F9FA
:1046F00093972700B307F9006308F70283A7040024
:1047000083A7C7022326F5028320C1010324810168
:1047100083244101032901018329C10013010102FE
:1047200067800000678000009309450013040500BE
:1047300013850900EFC04F8A83A7040017C7010043
:10474000130747E20327070083A7C7022326F402C3
:104750006376F70017C701002326F7E013952700BB
:104760003305F50003248101131525008320C101C1
:1047700083244101938509003305A9008329C100E1
:1047800003290101130101026FB0DFFC630605027A
:10479000130101FF2326110023248100232291000D
:1047A00097C70100938787DD03A40700630AA4006D
:1047B000737004306F000000130500006780000074
:1047C0008327440563960700737004306F00000070
:1047D0008326C402032704059387F7FF232AF404E2
:1047E0006384E600638E0700130500008320C10088
:1047F000032481008324410013010101678000002C
:104800009304440013850400EFB01FFD0325040545
:1048100097C70100938707D503A7070093075000A8
:10482000B387A7402326A402232CF4006376A700B5
:1048300097C7010023A8A7D293054001EF40C018F5
:1048400097C701009387C7E33385A70093850400CA
:10485000EFB05FF0130510006FF05FF97370043074
:1048600097C701009387C7CF83A70700638007021C
:1048700097C70100938787D003A7070083A7070086
:1048800083274704938717002322F70467800000DB
:1048900097C701009387C7CC83A70700638C0702E3
:1048A00097C70100938787CD03A707000327470415
:1048B0006302070203A7070083A6070083274704B4
:1048C0009387F7FF2322F70483A746046394070026
:1048D000736004306780000097C70100938707CAA0
:1048E00003A6070083A6070003A70700930750004D
:1048F00083A6C60203258601B387D740232CF70081
:104900006780000097C70100938747C703A7070088
:10491000630A070083A6070003A7460513071700CD
:1049200023AAE60403A5070067800000130101FD28
:104930002320210323261102232481022322910212
:10494000232E3101130905007370043097C4010050
:10495000938404C183A7040017C40100130404C294
:10496000639E070A8327040083A78705639A0700CD
:10497000832704001307100023AEE704639A050E93
:1049800083A70400638807008327040083A74704E4
:10499000639A07147370043083A7040063940706B6
:1049A0008327040003A58705630805006302090443
:1049B0008327040023AC07048327040023AE0704E5
:1049C00083A70400638807008327040083A74704A4
:1049D000639207068320C1020324810283244102DB
:1049E000032901028329C10113010103678000002B
:1049F00003270400832787059387F7FF232CF704F9
:104A00006FF09FFB032704008327040083274704DC
:104A1000938717002322F7046FF09FF80327040001
:104A20008327040083274704938717002322F70472
:104A30006FF05FF3032704008326040083274704F5
:104A40009387F7FF2322F70483A74604E39407F82C
:104A5000736004308320C102032481028324410255
:104A6000032901028329C1011301010367800000AA
:104A7000032504002326B10013054500EFB0DFD560
:104A80008325C1009307F0FF6380F50897C70100F5
:104A9000938787AD83A907000327040083A7070036
:104AA000B389B9002322370163ECF90697C70100E7
:104AB000938787AC03A507008325040093854500F1
:104AC000EFB05FCC97C70100938747A883A7070083
:104AD00063F6F90097C7010023AA37A7EFB05FABD1
:104AE0006FF01FEA0327040083260400832747048E
:104AF0009387F7FF2322F70483A74604E39C07E884
:104B0000736004306FF01FE98325040017C50100AE
:104B1000130545C293854500EFB0DFC36FF01FFC5E
:104B200097C70100938707A503A507008325040005
:104B300093854500EFB01FC56FF05FFA130101FDCB
:104B400023202103232E3101232611022324810255
:104B500023229102232C41011389050093090600A9
:104B60007370043097C401009384849F83A704006A
:104B700017C40100130484A0639C071403270400D6
:104B8000930720000327C7056304F7028327040067
:104B90001345F5FF03A787053375E50023ACA7048C
:104BA000832704001307100023AEE704639A060A64
:104BB00083A70400638807008327040083A74704B2
:104BC000639407167370043083A70400639E07067E
:104BD000638809008327040083A7870523A0F900C1
:104BE0000327040093071000130500000327C705DF
:104BF000630EF700832704001349F9FF1305100023
:104C000003A787053379E90023AC27058327040030
:104C100023AE070483A704006388070083270400EA
:104C200083A747046392070C8320C10203248102F7
:104C300083244102032901028329C101032A81013E
:104C40001301010367800000032704008327040089
:104C500083274704938717002322F7046FF05FF739
:104C6000032504002326D10013054500EFB0DFB66D
:104C70008326C1009307F0FF638AF60C97C70100F3
:104C80009387878E03AA07000327040083A70700E2
:104C9000330ADA00232247016368FA0C97C7010040
:104CA0009387878D03A5070083250400938545001E
:104CB000EFB05FAD97C701009387478983A70700CF
:104CC0006370FA0A97C7010023A247896F00400961
:104CD00003270400832704008327470493871700D2
:104CE0002322F7046FF09FE90327040083260400C2
:104CF000832747049387F7FF2322F70483A74604FB
:104D0000E39407F2736004308320C102032481021C
:104D100083244102032901028329C101032A81015D
:104D200013010103678000000327040083260400A9
:104D3000832747049387F7FF2322F70483A74604BA
:104D4000E39207E8736004306FF0DFE78325040027
:104D500017C501001305059E93854500EFB09F9F81
:104D6000EFB01F836FF0DFE497C701009387878060
:104D700003A507008325040093854500EFB09FA09D
:104D80006FF01FFE630A050C130101FF23261100BB
:104D900023248100232291002320210173700430F9
:104DA00097B401009384C47B83A70400639607082B
:104DB000638606008327850523A0F6009307060077
:104DC000930620000326C505232ED504138705006E
:104DD000130405006382D70A63F4F60893053000D4
:104DE0006388B700930540006396B700630CD61044
:104DF000232CE40493071000630CF608130410003E
:104E000083A70400638C070097B701009387077797
:104E100083A7070083A747046398070613050400C8
:104E20008320C10003248100832441000329010061
:104E3000130101016780000097B701009387077491
:104E400003A7070083A7070083274704938717005A
:104E50002322F7046FF0DFF5737004306F00000059
:104E600093061000E398D7F88327850533E7B7004A
:104E7000232CE5046FF01FF883278505938717001F
:104E8000232CF5046FF01FF7EFD00FA36FF01FF97D
:104E90001309440013050900EFB01F9497B70100F0
:104EA0009387476C0325C40283A7070063F6A70016
:104EB00097B7010023A8A76A93054001EF30D030CF
:104EC00097B701009387C77B3385A7009305090037
:104ED000EFB05F8883278402638607007370043015
:104EE0006F00000097B701009387476983A7070009
:104EF0000327C40283A7C702E3F2E7F0EFB04FE94C
:104F00006FF0DFEF130400006FF09FEF63080508F8
:104F1000130101FE232C8100232A91002328210163
:104F2000232631012324410123225101232E110084
:104F300093090700138A06009304060013890500ED
:104F400013040500EFB00FF9930A050063060A0089
:104F5000832784052320FA000327C4059307200034
:104F6000232EF4046380F40463FA97109306300050
:104F70006388D400930640006396D400630CF70E58
:104F8000232C2405930710006312F70A8327840259
:104F900063820702737004306F0000007370043086
:104FA0006F0000008327840593871700232CF404E7
:104FB0006FF05FFD97B701009387075983A707003C
:104FC0006390070A9304440013850400EFB0DF8068
:104FD00097B70100938707590325C40283A70700E9
:104FE00063F6A70097B7010023AEA75693054001CB
:104FF000EF30901D97B70100938787689385040071
:105000003385A700EFB00FF597B7010093870757D7
:1050100083A707000327C40283A7C70263F8E7003A
:10502000638609009307100023A0F9001304100001
:1050300013850A00EFB08FE9130504008320C10136
:105040000324810183244101032901018329C10033
:10505000032A8100832A41001301010267800000B6
:105060009305840117B501001305456AEFB08FEE73
:105070006FF09FF9130400006FF09FFB930710007F
:10508000E392F4F08327840533E92701232C2405D8
:105090006FF05FEF630A050E130101FE232C810000
:1050A000232A91001304050023263101232E110029
:1050B0002328210193840500EFB0CFE1930720005E
:1050C0008326C405232EF4048327840513071000C8
:1050D0009309050093871700232CF4046396E608D0
:1050E0008327840263860700737004306F0000001A
:1050F00097B701009387474583A70700639A07087E
:105100001309440013050900EFB00FED97B7010034
:10511000938747450325C40283A7070063F6A700CA
:1051200097B7010023A0A74493054001EF30D009B1
:1051300097B701009387C754930509003385A700EB
:10514000EFB04FE197B701009387474383A707006C
:105150000327C40283A7C70263F8E700638604003D
:105160009307100023A0F400032481018320C101D0
:105170008324410103290101138509008329C1000A
:10518000130101026FB08FD4737004306F00000000
:105190009305840117B5010013054557EFB08FDB68
:1051A0006FF05FFA9307050063080506737004301B
:1051B00017B701001307C73A83260700639E06024C
:1051C00003A6C70593062000130500006316D6004A
:1051D00023AE07041305100083270700638C070024
:1051E00097B701009387873903A707000327470470
:1051F000631C07026780000097B60100938606389B
:1052000003A6060083A6060083264604938616009E
:105210002322D6046FF0DFFA97B701009387073691
:1052200083A707006FF09FF803A7070083A6070076
:10523000832747049387F7FF2322F70483A74604B5
:10524000E39A07FA7360043067800000130101FBE2
:105250002322910423202105232C4103232A5103D7
:1052600023286103232671032326110423248104A8
:10527000232E310323248103232291032320A1031E
:1052800017B901001309893017BB0100130B4B2F0D
:1052900097B401009384042F97BA0100938ACA2E11
:1052A000130A1000930B90008327090003A707003F
:1052B0006306071683A7C70083A90700EFD0DFCFD7
:1052C000EFD01FD183270B00130C05006368F50C8A
:1052D00097B7010023A6A72A13060000637635239B
:1052E00003A50400B3858941EFC05FC0EFE04F80A4
:1052F0006306051603A504009306000013060000CC
:1053000093058100EFC0CFBEE30005FA832781003B
:10531000E3C207FE8329010183A7490163860700D1
:1053200013854900EFB04FCBEFD09FCA83270B0006
:10533000130C05006362F50C8327810017B7010089
:1053400023208725E3E8FBFAB317FA0013F70721B8
:105350006310072013F7770C6316072A93F70702E9
:10536000E38A07F813850900EF00504F6FF09FF8AC
:1053700083A7C70003A4C70083AC070093094400B8
:1053800013850900EFB04FC58327440213050400BD
:10539000E78007008327C4016386470D8327090040
:1053A00003A70700E31607FC03A70A0097B601004E
:1053B00023A8861D97B6010023A8F61C97B7010005
:1053C00023A6E71CEFD0DFF26FF0DFF283A7C70060
:1053D00003A4C70003AD0700930C440013850C0021
:1053E000EFB08FBF8327440213050400E780070056
:1053F0008327C401638C470B8327090003A7070099
:10540000E31607FC03A70A0097B6010023AEF616C1
:1054100097B7010023ACE7166FF01FF2EFD0DFB9AA
:10542000EFD01FBB83270B00130C0500E368F5F6D4
:1054300083A70A0003A504009309000003A6070040
:10544000B385894117B70100232C87131336160043
:10545000EFC0DFA9EFD0DFE9E31E05E8EFB04F931F
:105460006FF05FE98327840193850900B387FC000F
:1054700063E2FC0883A7040063860702232A010075
:10548000232C9101232E8100EFF08F9D03A50400B2
:10549000930600001306000093054101EFB00FEBE7
:1054A000E31E05EE737004306F0000008327840153
:1054B00093850C00B307FD006362FD0883A7040019
:1054C00063860702232A0100232CA101232E8100D9
:1054D000EFF00F9903A504009306000013060000E7
:1054E00093054101EFB08FE6E31805F073700430C7
:1054F0006F000000032509002322F4002328840004
:10550000EFB04FA86FF09FE9EFD09FDE832709002F
:1055100083A7C70003A4C700930C440013850C00A5
:10552000EFB08FAB8327C401638A4705832744020A
:1055300013050400E78007006FF0DFDB0325090097
:105540002322F40023288400EFB0CFA36FF0DFEA1A
:105550008327C10023ACF9006382070AB387870160
:1055600023A2F90023A83901938549006362FC084E
:1055700003A50A00EFB00FA16FF0DFD783278401E6
:10558000232884003387F9002322E400636AEC04B3
:10559000330C3C41636EFC0283A704006386070260
:1055A000232A0100232C3101232E8100EFF04F8BA1
:1055B00003A50400930600001306000093054101B3
:1055C000EFB0CFD8E31405F6737004306F0000001D
:1055D00003A50A0093850C00EFB0CF9A6FF01FF57A
:1055E0000325090093850C00EFB0CF996FF01FF4ED
:1055F00003250900EFB00F996FF0DFCF737004300F
:105600006F0000008327C10083A6890123A8390108
:105610003387D70023A2E9006362EC06B307FC409E
:1056200063EAD70683A7490213850900E7800700CC
:1056300083A7C901E39047CD83A689018327C100D1
:1056400003A70400B387D70063060702232A0100DB
:10565000232CF100232E3101EFF08F8003A50400ED
:10566000930600001306000093054101EFB00FCE32
:10567000E31205C8737004306F0000006374FC000F
:10568000E372F7FA0325090093854900EFB08F8F85
:105690006FF05FC603A50A0093854900EFB08F8EB7
:1056A0006FF05FC5130101FF232481002326110041
:1056B000232291002320210117B40100130484EC5C
:1056C000EFF0CF998327040063840704EFF04F9C29
:1056D00083270400638A0702930800001308000070
:1056E00093070000130720009306000013060040F4
:1056F00097B50100938585CC17050000130545B5C6
:10570000EFC05F9E63140506737004306F000000E5
:1057100017B901001309490313050900EFB00F8100
:1057200097B401009384840313850400EFB00F80C5
:10573000130600009305C0001305400097B7010051
:1057400023A627E597B7010023A097E4EFB0CFABDE
:1057500017B701002328A7E26306050297B50100E9
:10576000938545C5EFC04FE56FF05FF68320C1001C
:105770000324810083244100032901001301010156
:1057800067800000737004306F000000638A050AB0
:10579000130101FD232A5101930A05001305C002DC
:1057A000232481022322910223202103232E31016D
:1057B000232C410123261102232861012326710194
:1057C0001309070093890600130A06009384050055
:1057D000EF00C07013040500630C0502EFF00F88A2
:1057E00097B70100938707DA83A70700638E070442
:1057F000EFF00F8A1305440023205401232C94005A
:10580000232E44012320340323222403EFA01FF47A
:10581000130504008320C102032481028324410272
:10582000032901028329C101032A8101832A41013D
:10583000032B0101832BC1001301010367800000CA
:10584000737004306F00000097BB0100938BCBEFA7
:1058500013850B00EFA09FED17BB0100130B0BF09E
:1058600013050B00EFA09FEC130600009305C0008A
:105870001305400097B7010023AA77D197B701001D
:1058800023A467D1EFB04F9817B70100232CA7CE00
:10589000630A050097B501009385C5B1EFC0CFD16C
:1058A0006FF01FF5737004306F000000630E050683
:1058B000130101FE232C8100232E1100232A9100C5
:1058C00017B40100130404CC832804001308050056
:1058D0001305000063800804930407002322B1002D
:1058E000138706002324C1002326010193065000DC
:1058F00063C0B604EFE0DFD693072000630EF50423
:1059000003250400930600001306000093054100E0
:10591000EFB0CFA38320C10103248101832441017F
:105920001301010267800000737004306F000000F3
:105930009305410093060000130607001385080035
:10594000EFB05FAD8320C1010324810183244101B5
:105950001301010267800000032504009306000084
:105960001386040093054100EFB04F9E6FF09FFA3D
:10597000630605000325050067800000737004308E
:105980006F00000063160500737004306F000000A4
:10599000130101FF232611002324810013040500B5
:1059A000EFE0DFEB032544013334A000EFE05FEECE
:1059B000130504008320C1000324810013010101A9
:1059C0006780000063160500737004306F000000EC
:1059D000130101FF23248100130405002326110075
:1059E000EFE0DFE703240402EFE09FEA8320C10039
:1059F00013050400032481001301010167800000E6
:105A000063160500737004306F000000130101FF7E
:105A100023248100232291001384050093040500B0
:105A200023261100EFE09FE323A0840203248100DA
:105A30008320C10083244100130101016FE05FE571
:105A4000130101FF1305C001232481002326110047
:105A5000EF00C0481304050063080500232005007B
:105A600013054500EFA09FCC130504008320C1005F
:105A70000324810013010101678000006302050215
:105A8000B70700FFB3F7F5006386070073700430B3
:105A90006F000000639A0500737004306F0000000F
:105AA000737004306F000000130101FE232C81008D
:105AB00023282101232631012324410123225101DE
:105AC000232E1100232A9100930907001389060051
:105AD000930A060013840500130A0500EFE05FB87F
:105AE0006318050063860900737004306F000000BE
:105AF000EFD08FCC83240A00B3779400631209049B
:105B00006382070463880A009347F4FFB3F79700A2
:105B10002320FA00EFD0CFFD8320C10103248101AF
:105B20001385040003290101832441018329C10055
:105B3000032A8100832A41001301010267800000CB
:105B4000E302F4FCE38809FCB33550019395850129
:105B500063060900B7070004B3E5F50013860900E2
:105B6000B3E5850013054A00EFE0CFE1EFD04FF831
:105B700063140500EFA0DFA1EFE01FD693176500C7
:105B80009309050063DA0700B70400019384F4FF6A
:105B9000B3F499006FF05FF8EFE05FCC83290A005F
:105BA000B377340163100902638A070063880A002F
:105BB0009347F4FFB3F737012320FA00EFE05FCDFE
:105BC0006FF09FFCE31CF4FE6FF05FFE630C0500BA
:105BD000B70700FFB3F7F500638A0700737004305E
:105BE0006F000000737004306F000000130101FFAC
:105BF0002324810013040500232611002322910091
:105C00002320210113890500EFE05FC583240400F0
:105C10009345F9FFB3F795002320F400EFE05FC749
:105C20008320C1000324810013850400032901009F
:105C3000832441001301010167800000130101FF6B
:105C4000232481001304050023261100EFA09FA840
:105C500003240400EFA09FA78320C10013050400C4
:105C6000032481001301010167800000630C05001B
:105C7000370700FFB3F7E500638A0700737004304D
:105C80006F000000737004306F0000006F205061DF
:105C9000B70700FFB377F600638607007370043020
:105CA0006F00000063160600737004306F00000080
:105CB000130101FE232C8100232821012326310119
:105CC00023244101232E1100232A91001389060069
:105CD00093890500130A050013040600EFE05F989E
:105CE000631E050463060900737004306F00000032
:105CF000EFD08FAC83240A009385090013050A00B6
:105D0000B3E49900EFF09FF6B3779400630AF408C8
:105D100083240A00EFD0CFDD8320C1010324810159
:105D20001385040003290101832441018329C10053
:105D3000032A81001301010267800000EFD0CFA782
:105D400083240A009385090013050A00B3E4340193
:105D5000EFF0DFF1B3F7840063848704E30A09FA04
:105D6000B705000513060900B365B40013054A0022
:105D7000EFE04FC1EFD0CFD763140500EFA05F81F4
:105D8000EFE09FB5931765009304050063D4070205
:105D9000B70700019387F7FFB3F4F4006FF0DFF764
:105DA00083270A001344F4FFB3F787002320FA0087
:105DB0006FF05FF6EFE09FAA83240A00B3779400A8
:105DC000639887009347F4FFB3F797002320FA0006
:105DD000EFE01FAC6FF0DFFB130101FF2324810014
:105DE000232611001304050023229100EFD0CF9C3D
:105DF0008327440063860702032504019304C4003B
:105E0000631895006F008003032504016308950261
:105E1000B7050002EFE04FE183274400E39607FE59
:105E200013050400EF008023032481008320C100B8
:105E300083244100130101016FD08FCB73700430B4
:105E40006F000000630C0500370700FFB3F7E500A3
:105E5000638A0700737004306F00000073700430B1
:105E60006F0000006F20D043630C0500B70700FFF0
:105E7000B3F7F500638A0700737004306F00000009
:105E8000737004306F000000130101FF23248100B0
:105E9000232291002326110013040500938405009A
:105EA000EFE0DF9B0327040093C7F4FFB377F7000D
:105EB0002320F400032481008320C10083244100B7
:105EC000130101016FE0DF9C6306050003258501D6
:105ED000678000001305000067800000130101FFC8
:105EE000232481002326110013040500EFD0CF8C5A
:105EF00097A701009387C76983A70700639C0704DE
:105F0000B797010017B701001307C7869387C7FF2C
:105F100097A6010023A4E66817A70100232EF766C1
:105F200017B70100232AF78497A701009387876694
:105F300017B701002320F7849307100017A701006B
:105F40002320076617A701002326076417A701006F
:105F50002320F76463120402EFD08FB9EF1080584A
:105F600013040000130504008320C10003248100F2
:105F70001301010167800000130584009377350049
:105F80006398070CB79701001307F5FF9387A7FFE6
:105F9000E3E4E7FC97A601009386466083A706002A
:105FA0006F00400103A70700630A070093860700FC
:105FB0009307070003A74700E366A7FE17A70100A2
:105FC0001307475DE38AE7F803A7070013060001FC
:105FD0001384870023A0E60003A74700B306A74069
:105FE000637ED6023388A7002322D80023A2A7000D
:105FF0008325480097A601009386465A6F008000CB
:106000009306070003A7060003264700E36AB6FECF
:106010002320E80023A0060103A7470097A701005B
:106020009387075B83A70700B387E74017A70100A3
:106030002320F75AEFD0CFABE30204F2130504009C
:106040008320C10003248100130101016780000047
:106050001375C5FF130545006FF0DFF263080506F1
:10606000130101FF232481002326110013040500DE
:10607000EFC09FF4930584FF0326C4FF17A7010018
:106080001307C7516F00800013870700832707009D
:1060900083A64700E3EAC6FE232CF4FE2320B700C4
:1060A00097A701009387C75203A707008327C4FF60
:1060B000032481008320C100B387E70017A70100F4
:1060C0002328F750130101016FD08FA267800000D1
:1060D00097A701009387C74F03A5070067800000BB
:1060E000678000003367B50013773700930705001A
:1060F000631207049308D6FFB308150113070500C0
:10610000938605006378150303A80600130747006C
:1061100093864600232E07FFE36817FF9347F5FF9A
:10612000B387170193F7C7FF93874700B385F5003F
:10613000B307F5003306C50063F4C70C938645002A
:1061400013884700B3B6D70033B8050133E7F5002D
:1061500093C616001348180013773700B3E60601FC
:10616000133717003377D700330EF64093861700A6
:10617000630807061337AE006314070613532E0097
:106180001388050093860700130700008328080082
:10619000130717001308480023A016019386460032
:1061A000E36667FE1377CEFFB385E500B387E700AC
:1061B0006306EE0483C60500138717002380D7000B
:1061C000637EC70283C6150013872700A380D7000C
:1061D0006376C70203C725002381E70067800000BC
:1061E000B307F640B387F5009385150003C7F5FFA5
:1061F00093861600238FE6FEE398F5FE6780000085
:1062000067800000B367C50093F73700B308C50087
:106210006382070E63761511B307A04093F737002A
:10622000138737009306500093F5F50F13081500F8
:106230003383A8401306F6FF6374D700130750009A
:106240006368E60E6380070E2300B5001307100095
:10625000638EE700A300B500130730001308250084
:106260006396E700130835002301B50013968500F7
:1062700033E6C500139705013367E6003303F340A7
:1062800093968501B366D70013562300B307F50034
:106290001307000023A0D7001307170093874700B8
:1062A000E36AC7FE1377C3FFB307E8006300E308A0
:1062B0002380B70013871700637C1703A380B70000
:1062C00013872700637617032381B70013873700EE
:1062D00063701703A381B70013874700637A170120
:1062E0002382B7001387570063741701A382B70096
:1062F0006780000093F5F50F13978500B365B7002D
:10630000139705013367B700E37415FF9307050082
:106310009387470023AEE7FEE3EC17FF678000009A
:1063200067800000130805006FF05FF467800000CD
:10633000930705006FF0DFF783470500130705009B
:10634000638C07001305150083470500E39C07FED7
:106350003305E540678000001305000067800000FA
:10636000130515008347F5FF9385150003C7F5FF57
:1063700063880700E386E7FE3385E7406780000017
:10638000930700006FF05FFF9307050093851500EA
:1063900003C7F5FF93871700A38FE7FEE31807FEF7
:1063A0006780000083460500930700026398F600AB
:1063B0001305150083460500E38CF6FE938756FD12
:1063C00093F7D70F63800704930705009305000038
:1063D000638806041305000093871700138606FDE3
:1063E0001317250083C607003305A70013151500F2
:1063F0003305A600E39206FE638405003305A04042
:1064000067800000938536FD8346150093B515001F
:1064100093071500E39006FC130500006FF0DFFD05
:10642000130500006780000083A705002380A700F4
:1064300083A705009387170023A0F500678000005D
:1064400097A601009386061683A706001737030058
:106450001307473313861700B307F7002380A700FD
:1064600097A5010023A0C5149307A000630AF500B7
:10647000930700046308F60013050000678000001E
:10648000E30C06FE370610F0130717008347F7FFEB
:106490002320F6F083A706009387F7FF97A5010056
:1064A00023A2F510E39207FE1305000067800000A9
:1064B000130101EB2322911423202115232A5113C8
:1064C000232481132326111423248114232E311312
:1064D000232C4113232861132326711323229113A4
:1064E0002320A113232EB111930405001389050065
:1064F0002326C100130C5002930A90008347090021
:1065000063888703638C070603A404006F00800080
:10651000638607062300F40003A40400130919008E
:106520001304140023A0840083470900E39287FF2B
:10653000034619009308190093860800130D000202
:106540009309F0FF130AF0FF13080000130550052C
:106550009307D6FD93F7F70F13891600636EF53A8C
:1065600017A70100130707AA93972700B387E7002F
:1065700083A70700B387E700678007008320C11463
:106580000324811483244114032901148329C11392
:10659000032A8113832A4113032B0113832BC11276
:1065A000032C8112832C4112032D0112832DC11162
:1065B0001301011567800000930C80002324010063
:1065C0009307100063DA071D8327C10003A40400AA
:1065D000938B770093F68BFF03AB060083A94600ED
:1065E000938786002326F10013860C009306000093
:1065F00013050B0093850900EF10106D2328A100EF
:106600009307000063803733930D4101930B100013
:1066100013860C009306000013050B0093850900F8
:10662000EF10D00C9306000013860C00130B05002E
:1066300093890500EF1050698327810023A0AD00E6
:1066400093861B00938D4D0063863701938B060064
:106650006FF01FFCE37C9BFF63D2460393070400AB
:106660002380A70103A40400130AFAFF9307140070
:1066700023A0F40013840700E3C446FF93962B0085
:1066800093070101B386D7006F00800293877705D7
:106690002300F40003A40400938BFBFF93871B00EB
:1066A0001304140023A084009386C6FFE358F0E48B
:1066B00083A70600E3ECFAFC938707036FF05FFD06
:1066C00083A70400930600030327C1002380D7009B
:1066D00083A7040093064700930C0001138617005C
:1066E00023A0C40013068007A380C70003A40400EE
:1066F00023240100930707001304140023A084003F
:1067000003AB0700930900002326D1006FF0DFEDF3
:106710008327C10083AC0700938B470063880C2854
:10672000635C40259307D002631EFD2083C70C00E5
:106730006388070263D8092483A60400938C1C0095
:10674000130AFAFF2380F60003A4040013041400C4
:1067500023A0840083C70C00E39E07FC6352400320
:1067600003A40400930700022300F40003A4040020
:10677000130AFAFF1304140023A08400E3160AFE90
:10678000232671016FF09FD7232401009307100087
:10679000930CA000E3CA07E38327C10003A404000D
:1067A000938647006FF0DFF503C6160093060900D5
:1067B0006FF01FDA83A70400930650022380D700EE
:1067C00003A404001304140023A084006FF01FD35B
:1067D000930C0001232401006FF09FDE8327C1008A
:1067E00003C616009306090083A907009387470094
:1067F0002326F100E35E0AD4138A09009309F0FF0F
:106800006FF01FD503C61600130DD00293060900C2
:106810006FF01FD49347FAFF93D7F74103C61600D2
:10682000337AFA00930609006FF09FD203C6160070
:10683000130D0003930609006FF09FD183C5160066
:10684000930906FD93060900938705FD138605004D
:10685000E3E2FAFA93972900B38937019386160089
:1068600093991900B389B90083C50600938909FD7E
:10687000938705FD13860500E3FEFAFC6FF09FF792
:106880000327C10083A704008326070013074700DE
:106890002326E1002380D70003A40400130414007E
:1068A00023A084006FF09FC59307100063D4070FE7
:1068B0008327C1009386770093F686FF938786002F
:1068C0002326F10083A9460083A7060063DE090E94
:1068D00083A604001306D002B307F0402380C6004D
:1068E00003A40400B336F000B309304113041400CC
:1068F00023A08400138B0700B389D940930CA00018
:10690000232401006FF05FCE03C6160013081800A1
:10691000930609006FF0DFC383A704001389080002
:106920006FF09FE9E3729BCF93071000930B000079
:1069300093061000E3C447D36FF05FD497AC010017
:10694000938C4CA89385090013850C00EF1040022E
:10695000330AAA406352400303A404002300A401A5
:1069600003A40400130AFAFF1304140023A08400F4
:10697000E3160AFE130A000083C70C00E38207E057
:10698000E3CC09DA9389F9FF1307F0FFE396E9DA1C
:106990006FF0DFDC8327C1009386470083A70700E1
:1069A0002326D10093D9F7416FF05FF2635640017F
:1069B0009307D002E314FDF897AC0100938C8CA0F0
:1069C000930780026FF01FD7138B0700930CA00072
:1069D0002324010003A404006FF01FC1130101EB85
:1069E000232E3113B70900409387F9FF2324811424
:1069F00023229114232C4113232A511323261114EB
:106A000023202115232861132326711323248113A6
:106A1000232291132320A113232EB111130A050061
:106A20002324B10017A401001304C4B7973A03004C
:106A3000938A4AD597940100938444722326F100E7
:106A4000930550021305A00013080004B70610F0C8
:106A500083470A00638EB7046388070A032704008C
:106A6000130A1A00130617003387EA0097A80100DB
:106A700023AAC8B22300F7006380A708E31A06FD23
:106A800017370300130707D0130717008347F7FFD3
:106A900023A0F6F0832704009387F7FF17A60100D1
:106AA0002322F6B0E39207FE83470A00E396B7FA83
:106AB00083461A0013051A0013070500930B000202
:106AC000130BF0FF130CF0FF1308000093055005A3
:106AD000930890009387D6FD93F7F70F130A1700DA
:106AE00063ECF54493972700B387970083A70700CB
:106AF000B38797006780070017370300130787C81D
:106B0000E31406F86FF0DFF48320C114032481142A
:106B100083244114032901148329C113032A8113F7
:106B2000832A4113032B0113832BC112032C8112DF
:106B3000832C4112032D0112832DC1111301011564
:106B400067800000930C8000130D00009307100075
:106B500063DA0721832781009387770093F787FF04
:106B600083AD070003AB4700138787002324E100B0
:106B700013860C009306000013850D0093050B008F
:106B8000EF1090142328A10063086D4513094101FB
:106B90009309100013860C009306000013850D0066
:106BA00093050B00EF10803413860C009306000051
:106BB000930D0500138B0500EF1010112320A90081
:106BC0009389190013094900E3166DFDE3F49DFD57
:106BD00013060004B70610F063D48903832704006A
:106BE00013871700B387FA0097A5010023ACE59A35
:106BF00023807701630AC706130CFCFFE3C089FFFB
:106C00008327C1001305C10093089000B386F900E3
:106C10009396260093070101B386D7001308A000BE
:106C200013030004370610F0E38CA6E083A70600E8
:106C30009305000363F4F80093057005032704002F
:106C4000B387B700930517003387EA0017AE01003A
:106C5000232ABE942300F70063860737638C6532CE
:106C60009386C6FF6FF05FFC17370300130787B1E9
:106C7000130717008347F7FF23A0F6F083270400CC
:106C80009387F7FF97A5010023AEF590E39207FEE7
:106C9000130CFCFF6FF09FF683270400130600041B
:106CA0001387170097A5010023AEE58EB386FA007F
:106CB000930500032380B6006308C750938727001D
:106CC00097A6010023A0F68E3387EA00930680077B
:106CD0002300D700173703001307C7AAB70610F021
:106CE0006392C702130717008347F7FF23A0F6F04C
:106CF000832704009387F7FF17A601002324F68A51
:106D0000E39207FE83278100930C0001130D00001E
:106D10009387470003278100130B0000832D070092
:106D20002324F1006FF0DFE48327810083AC0700A8
:106D300013894700638E0C4C6358802B9307D00255
:106D40006394FB3E03C70C00930507006314072AF6
:106D50006F00002F93071000930CA000130D00008C
:106D6000E3CA07DF83278100938747006FF09FFA0C
:106D7000832781008346170013070A0003AB07002F
:106D8000938747002324F100E3560CD4130C0B0027
:106D9000130BF0FF6FF01FD483461700930BD00244
:106DA00013070A006FF01FD39347FCFF93D7F741F7
:106DB00083461700337CFC0013070A006FF09FD155
:106DC00083461700930B000313070A006FF09FD050
:106DD00003461700138B06FD13070A00930706FDF1
:106DE00093060600E3E2F8FA93172B00B3876701D6
:106DF0001307170093971700B387C70003460700D0
:106E0000138B07FD930706FD93060600E3FEF8FCCF
:106E10006FF09FF783258100832704001306A000ED
:106E200003A7050093861700B387FA0017950100A2
:106E3000232AD5762380E700138945006300C736EF
:106E4000930700046384F62A232421016FF05FBFB7
:106E50009307100063DE07358327810013877700CF
:106E6000137787FF930787002324F100032B470044
:106E70008327070063560B3E032704001306000414
:106E8000930617009795010023AED5703387EA006B
:106E90009305D0022300B700638CC638B307F040D7
:106EA0003337F000330B6041938D0700330BEB4019
:106EB000930CA000130D00006FF09FCB83461700CA
:106EC0001308180013070A006FF0DFC0834617008D
:106ED00013070A006FF01FC0832704009306000405
:106EE0001387170017960100232EE66AB387FA006E
:106EF000130650022380C700E314D7B417370300EA
:106F000013074788B70610F0130717008347F7FFEA
:106F100023A0F6F0832704009387F7FF179601005C
:106F20002322F668E39207FE6FF09FB1930C0001F5
:106F3000130D00006FF09FC1832704009306000427
:106F4000130A05001387170017960100232CE66427
:106F5000B387FA00130650022380C700E312D7AEAE
:106F60001737030013070782B70610F0130717003F
:106F70008347F7FF23A0F6F0832704009387F7FFEA
:106F8000179601002320F662E39207FE130A05001C
:106F90006FF01FAB172703001307C77E13071700F7
:106FA0008347F7FF2320F6F0832704009387F7FF3A
:106FB0009795010023A8F55EE39207FE9386C6FF2E
:106FC0006FF09FC6172703001307C77BE39805FCE4
:106FD0009386C6FF6FF05FC5E3FA9DBB930910006F
:106FE0006FF01FBF130C000003C70C0093050700D0
:106FF000E30C07E49308F0FF1305A0001308000456
:10700000B70610F0635E0B0C83270400138617008D
:10701000B387FA00179301002326C3582380E700A3
:107020006382A5086308060B938C1C0003C70C0041
:10703000130CFCFF93050700E31607FCE35680E101
:10704000832704009305000213060004B70610F01E
:107050006F00C000130CFCFFE3080CDE1387170061
:10706000B387FA002380B70017950100232CE5525F
:1070700093070700E310C7FE172703001307877065
:10708000130717008347F7FF23A0F6F083270400B8
:107090009387F7FF179501002326F550E39207FE2B
:1070A0006FF05FFB172703001307C76DE30E06F6AB
:1070B000130717008347F7FF23A0F6F08327040088
:1070C0009387F7FF17960100232EF64CE39207FEF5
:1070D0006FF09FF5172703001307C76A6FF05FFD76
:1070E000130BFBFFE3121BF36FF05FF51727030091
:1070F00013074769B70610F0130717008347F7FF18
:1071000023A0F6F0832704009387F7FF179601006A
:10711000232AF648E39207FE232421016FF05F92B1
:10712000979C0100938C0C2A93050B0013850C008F
:10713000EF001004330CAC40E35880EB83270400CD
:1071400013060004B70610F06F00C000130CFCFF1C
:10715000E30A0CE813871700B387FA00238077014E
:107160009795010023A0E54493070700E310C7FEAD
:107170001727030013070761130717008347F7FF5B
:1071800023A0F6F0832704009387F7FF979501006B
:1071900023AAF540E39207FE6FF05FFB1727030079
:1071A0001307475EE39806F4232421016FF05F89FB
:1071B000832781001387470083A707002324E1006A
:1071C00013DBF7416FF01FCB172703001307875B13
:1071D000B70610F0130717008347F7FF23A0F6F058
:1071E000832704009387F7FF17960100232CF63AB4
:1071F000E39207FE93071000179701002324F73A44
:107200009307800717270300230EF7566FF09FAFF1
:10721000635680019307D002E394FBF0979C010032
:10722000938C4C1A13078002930580026FF09FDC49
:107230009726030093860655370610F093861600AE
:1072400003C7F6FF2320E6F0032704001307F7FF28
:107250009795010023A8E534E31207FE6FF01FC4E1
:10726000938D0700930CA000130D00006FF05F904A
:10727000B70710F023A0A7F26F000000130101FC74
:10728000130341022322B10293050300232E1100B0
:107290002324C1022326D1022328E102232AF1025A
:1072A000232C0103232E110323266100EFF00FF39B
:1072B0008320C10113050000130101046780000051
:1072C000130101FB13038103232481022326A10060
:1072D000232CC10213040500130603001305C1008B
:1072E000232611022322F104232ED1022320E104BC
:1072F0002324010523261105232E6100EFF04F9B67
:107300008327C100238007000325C1008320C10219
:1073100033058540032481021301010567800000C5
:10732000B70710F083A647F403A607F403A747F4B2
:10733000E31AD7FE9306067D33B6C600B305E60012
:1073400023A4D7F423A6B7F467800000B70710F092
:1073500003A747F403A607F483A647F4E31AD7FE6E
:107360009306067D33B6C60023A4D7F4B305E60022
:1073700023A6B7F49307000873A047306780000086
:10738000130101FF23248100232611009797010098
:107390009387C721179401001304042103A7070052
:1073A0008327040093064706938747061796010034
:1073B000232CF61EB7170000179601002328D61EAF
:1073C000938777BB63CAD7008320C1000324810061
:1073D0001301010167800000B7F7FFFF9387C74AD9
:1073E0003307F7009797010023A2E71CEF008043C3
:1073F000930710006316F50203270400B727000067
:107400009387773213050000E3D0E7FCEFF05FE6E7
:10741000032481008320C100130101016FB0DFB894
:1074200017950100130585FAEFF05FE513052000BD
:10743000EFF01FE4032481008320C1001301010148
:107440006FB09FB617950100130505FA6FF01FE3A3
:10745000179501001305C5F96FF05FE2130101FFF5
:10746000232481002322910023261100B714000059
:1074700017940100130444F8938784381300000024
:107480009387F7FFE39C07FE13050400EFF01FDF6F
:107490006FF09FFE130520006F000015130101FF20
:1074A00023261100EF000038130710009307000097
:1074B000631AE5008320C100138507001301010151
:1074C0006780000017950100130545F0EFF01FDB02
:1074D0008320C100930720001385070013010101D9
:1074E00067800000737004306F0000006780000048
:1074F000737004306F000000130101FE232C810023
:10750000232A910023282101232E110013040500B2
:107510002317010013090000930410006F0080007E
:1075200013091000032644000325040093060000FD
:107530009305E100EF905FB3E31495FE631E09002D
:107540000327840083570700938717009397070149
:1075500093D707412310F7008357E1009387170063
:107560002317F1006FF01FFC130101FD232481029A
:107570002322910223202103232E310123261102ED
:107580001304050093090000930400001309100080
:107590000326440003250400930600009305E10040
:1075A000EF909FCBE31625FF8357E1006388970098
:1075B00093840700930910006FF09FFD93841400DB
:1075C000639E0900032784008357070093871700F1
:1075D0009397070193D707412310F7009394040171
:1075E00093D404016FF0DFFA130101FE2326310169
:1075F000930905001305C000232E1100232C8100E0
:10760000232A910023282101EFE05F8D1304050058
:10761000130600009305200013051000EF90CFBE65
:107620001309803E97970100938707FA2320A4004F
:10763000232224012324F4001305C000EFE01F8A55
:107640009304050003250400138709009306040032
:1076500023A0A40017950100130585F623A4A40018
:107660009308000013080000930700001306004071
:1076700097950100938585D923A204001705000082
:107680001305C5EEEFA01FA6938604009308000023
:1076900013080000130700009307000013060040C2
:1076A00097950100938505D717050000130505E59B
:1076B000EFA05FA31305C000EFE05F821304050095
:1076C000130600009305200013051000EF90CFB3C0
:1076D000979701009387E7EE2320A4002324F4006A
:1076E000232204001305C000EFE04FFF93040500C0
:1076F000032504009306040023A2240123A0A40070
:1077000017950100130565EC23A4A400930800005D
:107710001308000093070000130700001306004041
:1077200097950100938585CF17050000130505E4A3
:10773000EFA05F9B13870900938604009308000065
:1077400013080000930700001306004097950100FE
:10775000938545CD17050000130545DAEFA09F98E6
:107760001305C000EFE08FF71304050013060000B7
:107770009305200013055000EF900FA99797010083
:10778000938747E42320A400232224012324F40028
:107790001305C000EFE08FF49304050003250400F7
:1077A0009306040023A2240123A0A400179501003E
:1077B0001305C5E123A4A4009308000013080000EA
:1077C000930700001307000013060040979501007F
:1077D0009385C5C517050000130545D2EFA09F90FE
:1077E000032481018320C101032901018329C100F0
:1077F00093860400832441019308000013080000CD
:10780000930700001307000013060040979501003E
:10781000938545C217050000130545D513010102E4
:107820006FA05F8C130101FF232221012326810019
:107830002324910023203101179501001305C5D899
:10784000179801001308C8D783540500835E05000C
:107850008359080017990100130989D5035E0800B0
:107860000354250083150900179701001307C7D497
:1078700003532500831707008353280003162700AE
:10788000939909018358280093D9094183524500EF
:107890009394040113140401035F45008316290027
:1078A000835F480093D40441B385354113540441A8
:1078B00003174700B387974033068640B335B000BF
:1078C0009393030103154900B305B04093D30341DB
:1078D000B337F0003336C00093920201B3F7B7001C
:1078E0003306C040B386764093D2024193950F0190
:1078F000B3F7C700B336D0000356480033075740EC
:1079000093D505410324C100B306D0403337E000CE
:107910003305B5403307E040B3F7D7003335A00057
:10792000B3F7E7003305A040179701002316D7C926
:1079300017970100231EC7C717970100231F67C6AB
:1079400017970100231717C7179701002318E7C7D8
:10795000179701002310C7C6832481000329410023
:107960008329010033F5A70013010101678000009E
:10797000B305B500930705006386B70003C707008A
:10798000631607003385A7406780000093871700C0
:107990006FF09FFE130101FB23229104232C41036E
:1079A000232291032326110423248104232021056B
:1079B000232E3103232A5103232861032326710335
:1079C000232481032320A103232EB101930C05005E
:1079D000138A05009304000063DE05003305A04010
:1079E0003337A000B305B040930C0500338AE5405F
:1079F0009304F0FF63DA06003306C040B337C000DB
:107A0000B306D040B386F640930A06009389060079
:107A100013840C0013090A0063960628179B0100C3
:107A2000130B4B896370CA16B70701006372F61413
:107A30009307F00F63F4C70093098000B357360132
:107A4000330BFB0083470B0013050002B38737019C
:107A5000B309F540638C0900B3153A01B3D7FC00B4
:107A6000B31A360133E9B70033943C0113DB0A0142
:107A700093050B0013050900EF00507C130A050065
:107A800093050B00939B0A0113050900EF00907604
:107A900093DB0B019305050013850B00EF00D072FB
:107AA000131A0A0193570401B367FA0063FAA70097
:107AB000B387570163E6570163F4A700B387570103
:107AC0003389A74093050B0013050900EF001077D9
:107AD000130A050093050B0013050900EF009071D0
:107AE0001314040193050500131A0A0113850B00F2
:107AF00013540401EF00506D33648A00637AA400CC
:107B000033045401636654016374A40033045401C4
:107B10003304A4403354340193050000638A040005
:107B200033048040B3378000B305B040B385F540DF
:107B3000130504008320C104032481048324410429
:107B4000032901048329C103032A8103832A4103F2
:107B5000032B0103832BC102032C8102832C4102DE
:107B6000032D0102832DC10113010105678000006F
:107B7000B707000193090001E362F6EC9309800165
:107B80006FF0DFEB631A0600930500001305100089
:107B9000EF005066930A0500B707010063FAFA0E7A
:107BA0009307F00F63F4570193098000B3D73A01AC
:107BB000330BFB0083470B001305000233095A41C6
:107BC000B3873701B309F540E38209EAB39A3A0172
:107BD000335BFA00B3153A01B3D7FC0093DB0A011B
:107BE00033E9B70013050B0093850B00EF00106518
:107BF000130A050093850B00139C0A0113050B0063
:107C0000EF00505F135C0C019305050013050C0099
:107C1000EF00905B131A0A0193570901B367FA004A
:107C200033943C0163FAA700B387570163E6570119
:107C300063F4A700B3875701338BA74093850B00EC
:107C400013050B00EF00905F130A050093850B00EE
:107C500013050B00EF00105A9305050013050C00E7
:107C6000EF00905693160901131A0A0193D60601E4
:107C7000B366DA0063FAA600B386560163E65601DE
:107C800063F4A600B38656013389A6406FF01FDE69
:107C9000B707000193090001E3EAFAF093098001B4
:107CA0006FF0DFF06376DA0093050A006FF01FE7EC
:107CB000B707010063FAF604930BF00F33B5DB004E
:107CC0001315350033D7A600978701009387875E89
:107CD000B387E70083CB070093050002B38BAB00AB
:107CE000338B7541631C0B0263E4460163EACC00ED
:107CF0003384CC40B306DA4033B98C003389264153
:107D0000930509006FF09FE1B7070001130500011B
:107D1000E3EAF6FA130580016FF0DFFAB396660125
:107D2000335D7601336DDD00B35D7A01B3156A0111
:107D300033DC7C0113540D01336CBC0013850D0042
:107D400093050400B3196601EF00504F930A050034
:107D50009305040013850D0033996C01931C0D01EC
:107D6000EF00504993DC0C01130A05009305050050
:107D700013850C00EF005045939A0A0113570C012C
:107D800033E7EA00930D0A00637EA7003307A701DB
:107D9000930DFAFF6368A7016376A700930DEAFFCE
:107DA0003307A701330AA7409305040013050A000F
:107DB000EF00D04893050400930A050013050A005C
:107DC000EF005043930505001304050013850C00D4
:107DD000EF00903F93150C01939A0A0193D505018A
:107DE000B3E5BA001307040063FEA500B385A5013F
:107DF0001307F4FF63E8A50163F6A5001307E4FF8A
:107E0000B385A501939D0D01B70C0100B3EDED0005
:107E10001384FCFFB3F78D0033F48900338AA54047
:107E200013850700930504002326F10093DD0D015F
:107E3000EF00903993050400930A050013850D00A7
:107E4000EF00903813DC090193050C002324A100F6
:107E500013850D00EF0050378327C10013040C0079
:107E600093050400130C050013850700EF00D035BF
:107E70008326810013D70A013305D5003307A700F5
:107E80006374D700330C9C01B70701009387F7FF99
:107E9000935507013377F70013170701B3F7FA007B
:107EA000B3858501B307F7006366BA00631EBA00A5
:107EB000637CF90033863741B3B7C700B385A5416A
:107EC000B385F54093070600B307F9403339F9004D
:107ED000B305BA40B385254133947501B3D7670123
:107EE0003364F400B3D565016FF05FC3130101FD86
:107EF00023229102232A51012326110223248102E5
:107F000023202103232E3101232C41012328610149
:107F10002326710123248101232291012320A10121
:107F2000930A050093840500639E06381304060037
:107F300093090500178901001309C93763F8C512B1
:107F4000B7070100138B05006378F6101307F00FD5
:107F50003337C70013173700B357E6003309F9006A
:107F6000834609003387E60093060002B386E640A5
:107F7000638C0600B394D40033D7EA003314D600E0
:107F8000336B9700B399DA00935A040193850A0082
:107F900013050B00EF00902A1309050093850A00D2
:107FA000931B040113050B00EF00D02493DB0B019E
:107FB000930405009305050013850B00EF00D02006
:107FC0001319090193D70901B367F900138A040053
:107FD00063FEA700B3878700138AF4FF63E8870076
:107FE00063F6A700138AE4FFB3878700B384A74032
:107FF00093850A0013850400EF005024130905003F
:1080000093850A0013850400EF00D01E939909019F
:1080100093040500930505001319090113850B004E
:1080200093D90901EF00501AB3693901138604008E
:1080300063FCA900B30934011386F4FF63E68900E9
:1080400063F4A9001386E4FF13140A013364C40027
:10805000130A00006F000013B707000113070001A7
:10806000E36CF6EE130780016FF01FEF138A060032
:10807000631A06009305000013051000EF00901727
:1080800013040500B7070100637EF4129307F00F95
:1080900063F48700130A8000B35744013309F900E1
:1080A000034709009306000233074701B386E64001
:1080B00063940612B3848440130A1000135B040116
:1080C00093050B0013850400EF00501713090500FA
:1080D00093050B0013850400931B0401EF0090111E
:1080E00093DB0B01930405009305050013850B003A
:1080F000EF00900D1319090193D70901B367F90037
:10810000938A040063FEA700B3878700938AF4FF75
:1081100063E8870063F6A700938AE4FFB3878700CC
:10812000B384A74093050B0013850400EF001011E2
:108130001309050093050B0013850400EF00900B55
:10814000939909019304050093050500131909018A
:1081500013850B0093D90901EF001007B3693901AA
:108160001386040063FCA900B30934011386F4FFED
:1081700063E6890063F4A9001386E4FF13940A01FF
:108180003364C4001305040093050A008320C10270
:108190000324810283244102032901028329C101AE
:1081A000032A8101832A4101032B0101832BC10092
:1081B000032C8100832C4100032D010013010103D6
:1081C00067800000B7070001130A0001E366F4ECC2
:1081D000130A80016FF05FEC3314D40033DAE4004B
:1081E000B399DA0033D7EA00935A0401B394D40068
:1081F00093850A0013050A00336B9700EF00100403
:108200001309050093850A0013050A00931B040156
:10821000EF00407E93DB0B019304050093050500FE
:1082200013850B00EF00407A1319090113570B0156
:108230003367E900138A0400637EA70033078700D1
:10824000138AF4FF636887006376A700138AE4FF4C
:1082500033078700B304A74093850A001385040001
:10826000EF00C07D1309050093850A001385040003
:10827000EF004078930405009305050013850B007B
:10828000EF00807413170B0113570701131909012D
:10829000B367E9001387040063FEA700B387870074
:1082A0001387F4FF63E8870063F6A7001387E4FFF2
:1082B000B3878700131A0A01B384A740336AEA0020
:1082C0006FF0DFDF63ECD51EB707010063F4F6043F
:1082D0001307F00FB335D7009395350033D7B600A9
:1082E00097870100938707FDB387E70003C707005F
:1082F000130A00023307B700330AEA4063160A0282
:1083000013041000E3E096E833B6CA0013441600E5
:108310006FF05FE7B707000193050001E3E0F6FCAB
:10832000930580016FF09FFBB35CE600B3964601B6
:10833000B3ECDC0033D4E40093DB0C01B3974401CD
:1083400033D7EA0093850B0013050400336BF70065
:10835000B3194601EF00806E1309050093850B00E9
:1083600013050400139C0C01EF00C068135C0C01A2
:10837000930405009305050013050C00EF00C0648D
:108380001319090113570B013367E9001384040023
:10839000637EA700330797011384F4FF6368970196
:1083A0006376A7001384E4FF33079701B304A74063
:1083B00093850B0013850400EF0040681309050046
:1083C00093850B0013850400EF00C0629304050041
:1083D0009305050013050C00EF00005F93170B01D8
:1083E0001319090193D70701B367F9001386040035
:1083F00063FEA700B38797011386F4FF63E8970134
:1084000063F6A7001386E4FFB387970113140401F2
:10841000B70B01003364C4001389FBFF337D2401D3
:1084200033F92901B384A7409305090013050D0012
:10843000EF008059935C040193050900130B0500BC
:1084400013850C00EF00405893D90901130C050067
:108450009385090013850C00EF00005713090500F0
:108460009385090013050D00EF00005633058501C3
:1084700093570B013385A700637485013309790194
:1084800093570501B387270163E6F402E392F4BC36
:10849000B70701009387F7FF3375F5001315050142
:1084A000337BFB0033964A0133056501130A000054
:1084B000E37AA6CC1304F4FF6FF09FB9130A00000F
:1084C000130400006FF01FCC130101FB232481046F
:1084D00023229104232E3103232291032326110406
:1084E00023202105232C4103232A51032328610340
:1084F00023267103232481032320A103232EB1010A
:10850000930C05009389050013040500938405006E
:10851000639E062613090600138A0600978A010047
:10852000938A4AD963F4C514B70701006376F6123B
:108530009307F00F63F4C700130A8000B357460196
:10854000B38AFA0003C70A00130500023307470184
:10855000330AE540630C0A00B395490133D7EC00B8
:1085600033194601B364B70033944C01935A09019F
:1085700093850A0013850400EF00404C9309050021
:1085800093850A00131B090113850400EF00804640
:10859000135B0B019305050013050B00EF00C042B0
:1085A0009399090193570401B3E7F90063FAA7000F
:1085B000B387270163E6270163F4A700B387270188
:1085C000B384A74093850A0013850400EF00004799
:1085D0009309050093850A0013850400EF0080418C
:1085E00013140401930505009399090113050B0069
:1085F00013540401EF00403D33E48900637AA40082
:1086000033042401636624016374A4003304240149
:108610003304A44033554401930500008320C10472
:108620000324810483244104032901048329C10311
:10863000032A8103832A4103032B0103832BC102F5
:10864000032C8102832C4102032D0102832DC101E1
:108650001301010567800000B7070001130A00013C
:10866000E36EF6EC130A80016FF05FED631A06000B
:108670009305000013051000EF00C0371309050033
:10868000B7070100637AF90E9307F00F63F427012F
:10869000130A8000B3574901B38AFA0003C70A00DE
:1086A00013050002B384294133074701330AE5402B
:1086B000E30E0AEA33194901B3DAE900B395490137
:1086C00033D7EC0093540901336BB70013850A00CC
:1086D00093850400EF00803693090500938504001C
:1086E000931B090113850A00EF00C03093DB0B01D7
:1086F0009305050013850B00EF00002D93990901E8
:1087000093570B01B3E7F90033944C0163FAA700C8
:10871000B387270163E6270163F4A700B387270126
:10872000B38AA7409385040013850A00EF00003147
:10873000930905009385040013850A00EF00802B40
:108740009305050013850B00EF00002893150B011E
:108750009399090193D50501B3E5B90063FAA50022
:10876000B385250163E6250163F4A500B3852501E2
:10877000B384A5406FF09FDFB7070001130A000123
:10878000E36AF9F0130A80016FF0DFF0E3E8D5E85F
:10879000B707010063FCF604930BF00F33B5DB0061
:1087A0001315350033D7A60097870100938787B04C
:1087B000B387E70083CB070093050002B38BAB00C0
:1087C000338B7541631E0B0263E4360163EACC0010
:1087D0003384CC40B386D94033B58C00B384A640F3
:1087E00013050400938504006FF05FE3B7070001F1
:1087F00013050001E3E8F6FA130580016FF09FFA14
:10880000B3966601335D7601336DDD0033D47901B3
:10881000B395690133DC7C0193540D01336CBC00CA
:108820001305040093850400B31A6601EF000021CC
:10883000130A0500938504001305040033996C01A5
:10884000931C0D01EF00001B93DC0C0113040500C9
:108850009305050013850C00EF000017131A0A0199
:1088600013570C013367EA00130A0400637EA70064
:108870003307A701130AF4FF6368A7016376A70013
:10888000130AE4FF3307A701B309A7409385040047
:1088900013850900EF00801A938504001304050076
:1088A00013850900EF0000159305050093040500EA
:1088B00013850C00EF00401193150C0113140401F3
:1088C00093D50501B365B4001387040063FEA500CA
:1088D000B385A5011387F4FF63E8A50163F6A5003E
:1088E0001387E4FFB385A501131A0A01B70C010031
:1088F000336AEA001384FCFFB3778A0033F48A00FA
:10890000B384A54013850700930504002326F100D6
:10891000135A0A01EF00400B930905009305040068
:1089200013050A00EF00400A13DC0A01930D05004D
:1089300093050C0013050A00EF0000098327C1000E
:10894000130A050093050C0013850700EF00C0070C
:108950003305B50113D709013307A7006374B701C5
:10896000330A9A01B70701009387F7FF9355070170
:108970003377F70013170701B3F7F900B385450103
:10898000B307F70063E6B400639EB400637CF900AC
:1089900033865741B3B7C700B385A541B385F540CA
:1089A00093070600B307F9403339F900B385B440A3
:1089B000B385254133947501B3D767013365F4005E
:1089C000B3D565016FF09FC51306050013050000C0
:1089D00093F61500638406003305C50093D5150092
:1089E00013161600E39605FE678000006340050637
:1089F00063C6050613860500930505001305F0FF01
:108A0000630C060293061000637AB6006358C00038
:108A10001316160093961600E36AB6FE13050000BF
:108A200063E6C500B385C5403365D50093D616000F
:108A300013561600E39606FE67800000938200003E
:108A4000EFF05FFB13850500678002003305A0404F
:108A500063D80500B305B0406FF0DFF9B305B0404F
:108A600093820000EFF01FF93305A04067800200F9
:108A70009382000063CA0500634C0500EFF09FF786
:108A80001385050067800200B305B040E35805FE7A
:108A90003305A040EFF01FF63305B04067800200B9
:108AA000130101FE232C8100232A910013040500E9
:108AB0009384050023282101232631012324410129
:108AC00023225101232E1100EFA00FCF8327040092
:108AD00003290401B7090001B3E59700930AC40014
:108AE0002320B400930400009389F9FF370A0002A1
:108AF0000327040063822A050326090013050900E1
:108B0000B3654701B37636019317560033F7E60095
:108B10000329490063C60700631607006FF05FFD75
:108B2000E398E6FC9317760063D40700B3E4D4001F
:108B3000EFB09F8F6FF0DFFB93C4F4FFB3F4E4005A
:108B400023209400EFA0CFFA032504008320C10165
:108B50000324810183244101032901018329C100E8
:108B6000032A8100832A410013010102678000006B
:108B7000130101FF13052000232611002324810087
:108B8000EFE09FA617E7FFFF1307C77F93060000DC
:108B9000130610009305400617850100130545864E
:108BA000EFC0DFBE6302050213040500EFA04FC251
:108BB000130605001307000093060000930510003C
:108BC00013050400EFC09FCEEFA08F8B8320C10060
:108BD00003248100130500001301010167800000D8
:02000004800278
:10000000A867FEFF1869FEFFB467FEFF1869FEFFD0
:100010001869FEFF1869FEFF1869FEFFDC67FEFF26
:100020001869FEFF1869FEFF0468FEFF1468FEFFF2
:100030001869FEFF2C68FEFF3C68FEFF3C68FEFF6F
:100040003C68FEFF3C68FEFF3C68FEFF3C68FEFF2C
:100050003C68FEFF3C68FEFF3C68FEFF1869FEFF3F
:100060001869FEFF1869FEFF1869FEFF1869FEFF98
:100070001869FEFF1869FEFF1869FEFF1869FEFF88
:100080001869FEFF1869FEFF1869FEFF1869FEFF78
:100090001869FEFF1869FEFF1869FEFF1869FEFF68
:1000A0001869FEFF1869FEFF1869FEFF1869FEFF58
:1000B0001869FEFF1869FEFF1869FEFF1869FEFF48
:1000C0001869FEFF1869FEFF1869FEFF1869FEFF38
:1000D0001869FEFF1869FEFF1869FEFF1869FEFF28
:1000E0001869FEFF1869FEFF1869FEFF1869FEFF18
:1000F0001869FEFF1869FEFF1869FEFF1869FEFF08
:100100008068FEFFA868FEFF1869FEFF1869FEFF01
:100110001869FEFF1869FEFF1869FEFF1869FEFFE7
:100120001869FEFF0869FEFF1869FEFF1869FEFFE7
:10013000B865FEFFC066FEFF1869FEFF1869FEFF86
:100140001067FEFF1869FEFF8867FEFF1869FEFF53
:100150001869FEFFD067FEFF746DFEFFE06DFEFFC5
:10016000806DFEFFE06DFEFFE06DFEFFE06DFEFFC7
:10017000E06DFEFF186CFEFFE06DFEFFE06DFEFF20
:10018000406CFEFF506CFEFFE06DFEFF686CFEFFF2
:10019000786CFEFF786CFEFF786CFEFF786CFEFFDB
:1001A000786CFEFF786CFEFF786CFEFF786CFEFFCB
:1001B000786CFEFFE06DFEFFE06DFEFFE06DFEFF80
:1001C000E06DFEFFE06DFEFFE06DFEFFE06DFEFF07
:1001D000E06DFEFFE06DFEFFE06DFEFFE06DFEFFF7
:1001E000E06DFEFFE06DFEFFE06DFEFFE06DFEFFE7
:1001F000E06DFEFFE06DFEFFE06DFEFFE06DFEFFD7
:10020000E06DFEFFE06DFEFFE06DFEFFE06DFEFFC6
:10021000E06DFEFFE06DFEFFE06DFEFFE06DFEFFB6
:10022000E06DFEFFE06DFEFFE06DFEFFE06DFEFFA6
:10023000E06DFEFFE06DFEFFE06DFEFFE06DFEFF96
:10024000E06DFEFFE06DFEFFE06DFEFFE06DFEFF86
:10025000E06DFEFFE06DFEFFBC6CFEFFF86CFEFF84
:10026000E06DFEFFE06DFEFFE06DFEFFE06DFEFF66
:10027000E06DFEFFE06DFEFFE06DFEFF646DFEFFD2
:10028000E06DFEFFE06DFEFFEC69FEFF406BFEFFE0
:10029000E06DFEFFE06DFEFFD06BFEFFE06DFEFF48
:1002A000FC6BFEFFE06DFEFFE06DFEFFD46DFEFF18
:1002B000000102020303030304040404040404040D
:1002C00005050505050505050505050505050505DE
:1002D00006060606060606060606060606060606BE
:1002E00006060606060606060606060606060606AE
:1002F000070707070707070707070707070707078E
:10030000070707070707070707070707070707077D
:10031000070707070707070707070707070707076D
:10032000070707070707070707070707070707075D
:10033000080808080808080808080808080808083D
:10034000080808080808080808080808080808082D
:10035000080808080808080808080808080808081D
:10036000080808080808080808080808080808080D
:1003700008080808080808080808080808080808FD
:1003800008080808080808080808080808080808ED
:1003900008080808080808080808080808080808DD
:1003A00008080808080808080808080808080808CD
:1003B000546D725100000000546D7220537663003A
:1003C000286E756C6C2900004572726F7220696E20
:1003D00020416C74426C636B51207461736B7320A9
:1003E0000D0A00006D69616F750A00006D69616F2B
:1003F00075320A0068756E6772790A004368656332
:100400006B54696D6572000051436F6E7342310029
:100410005150726F644232005150726F6442330027
:1004200051436F6E734234005150726F6442350015
:0804300051436F6E7342360068
:100438001000000000000000017A5200017C010158
:100448001B0D020050000000180000004075FEFF60
:100458005805000000440E507489039406990B81D6
:1004680001880292049305950796089709980A9AB5
:100478000C9B0D036C010AC144C844C944D244D33F
:1004880044D444D544D644D744D844D944DA44DB88
:10049800440E00440B0000004C0000006C000000FB
:1004A800447AFEFFDC05000000440E307089039595
:1004B8000781018802920493059406960897099883
:1004C8000A990B9A0C0370020AC144C844C944D261
:1004D80044D344D444D544D644D744D844D944DA40
:1004E800440E00440B00000050000000BC00000057
:1004F800D07FFEFF0005000000440E50748802897A
:10050800039305990B810192049406950796089721
:1005180009980A9A0C9B0D0320010AC144C844C9D2
:1005280044D244D344D444D544D644D744D844D9F7
:0C05380044DA44DB440E00440B000000D9
:0805CC00FC8F01000400000097
:040000058000004037
:00000001FF
